 SwiCEAux

 Timestamp is 540049cf (Fri Aug 29 17:37:19 2014)

 Preferred load address is 00100000

 Start         Length     Name                   Class
 0001:00000000 00012570H .text                   CODE
 0001:00012570 00000534H .text$yc                CODE
 0001:00012aa4 00000080H .text$yd                CODE
 0002:00000000 0000912cH .rdata                  DATA
 0002:0000912c 00000075H .rdata$debug            DATA
 0002:000091a4 000000c8H .xdata                  DATA
 0002:0000926c 00000034H .xdata$x                DATA
 0002:000092a0 00000000H ATL$__a                 DATA
 0002:000092a0 00000000H ATL$__z                 DATA
 0002:000092a0 0000003cH .idata$2                DATA
 0002:000092dc 00000014H .idata$3                DATA
 0002:000092f0 00000158H .idata$4                DATA
 0002:00009448 0000017aH .idata$6                DATA
 0002:000095d0 0000017cH .edata                  DATA
 0003:00000000 00000158H .idata$5                DATA
 0003:00000158 00000004H .CRT$XCA                DATA
 0003:0000015c 00000004H .CRT$XCAA               DATA
 0003:00000160 0000000cH .CRT$XCC                DATA
 0003:0000016c 0000005cH .CRT$XCL                DATA
 0003:000001c8 00000004H .CRT$XCU                DATA
 0003:000001cc 00000004H .CRT$XCZ                DATA
 0003:000001d0 00000004H .CRT$XIA                DATA
 0003:000001d4 00000004H .CRT$XIZ                DATA
 0003:000001d8 00000004H .CRT$XPA                DATA
 0003:000001dc 00000004H .CRT$XPZ                DATA
 0003:000001e0 00000004H .CRT$XTA                DATA
 0003:000001e4 00000004H .CRT$XTZ                DATA
 0003:000001e8 000001a0H .data                   DATA
 0003:00000388 000004c0H .bss                    DATA
 0004:00000000 000009b0H .pdata                  DATA
 0005:00000000 000000a0H .rsrc$01                DATA
 0005:000000a0 000003d0H .rsrc$02                DATA

  Address         Publics by Value              Rva+Base       Lib:Object

 0000:00000000       ___safe_se_handler_count   00000000     <absolute>
 0000:00000000       ___safe_se_handler_table   00000000     <absolute>
 0001:00000008       ??0CCEHWIntf@@QAA@XZ       00101008 f   CEHWIntf.obj
 0001:000002e4       ??1CCEHWIntf@@UAA@XZ       001012e4 f   CEHWIntf.obj
 0001:00000350       ?ConnectToBIOS@CCEHWIntf@@QAAJXZ 00101350 f   CEHWIntf.obj
 0001:00000a54       ?DisConnectFromBIOS@CCEHWIntf@@QAAXXZ 00101a54 f   CEHWIntf.obj
 0001:00000af4       ?StartListeningForEvents@CCEHWIntf@@QAAHP6AXPAUSwiNotifyVariant@@@Z@Z 00101af4 f   CEHWIntf.obj
 0001:00000b30       ?StopListeningForEvents@CCEHWIntf@@QAAXXZ 00101b30 f   CEHWIntf.obj
 0001:00000b50       ?GetHWAuxVersion@CCEHWIntf@@QAAXPADG@Z 00101b50 f   CEHWIntf.obj
 0001:00000c0c       ?SetHWPower@CCEHWIntf@@UAAJW4SWIHW_TYPE_Power@@@Z 00101c0c f   CEHWIntf.obj
 0001:00000d58       ?GetHWAudioPath@CCEHWIntf@@UAAHPAK@Z 00101d58 f   CEHWIntf.obj
 0001:00000f08       ?HWEnableAudio@CCEHWIntf@@UAAHH@Z 00101f08 f   CEHWIntf.obj
 0001:00000ffc       ?HWSetVolumnLevel@CCEHWIntf@@UAAHKK@Z 00101ffc f   CEHWIntf.obj
 0001:00001128       ?HWInitiateHostBoot@CCEHWIntf@@UAAHK@Z 00102128 f   CEHWIntf.obj
 0001:00001214       ?HWSetTetheredMode@CCEHWIntf@@UAAHHPAX@Z 00102214 f   CEHWIntf.obj
 0001:000012d8       ?HWSetDevicePowerState@CCEHWIntf@@UAAJKKK@Z 001022d8 f   CEHWIntf.obj
 0001:00001400       ?GetHWPower@CCEHWIntf@@UAAJPAW4SWIHW_TYPE_Power@@@Z 00102400 f   CEHWIntf.obj
 0001:000014fc       ??_ECCEHWIntf@@UAAPAXI@Z   001024fc f i CEHWIntf.obj
 0001:000014fc       ??_GCCEHWIntf@@UAAPAXI@Z   001024fc f i CEHWIntf.obj
 0001:0000153c       ??0CComCriticalSection@ATL@@QAA@XZ 0010253c f i CEHWIntf.obj
 0001:00001570       ??1CComCriticalSection@ATL@@QAA@XZ 00102570 f i CEHWIntf.obj
 0001:00001580       ?Term@CComCriticalSection@ATL@@QAAJXZ 00102580 f i CEHWIntf.obj
 0001:000015ac       ?_AtlRaiseException@ATL@@YAXKK@Z 001025ac f i CEHWIntf.obj
 0001:000015d0       ??0CHWIntf@@QAA@XZ         001025d0 f   HWIntf.obj
 0001:00001694       ??1CHWIntf@@UAA@XZ         00102694 f   HWIntf.obj
 0001:00001764       ?NotifyCallback@CHWIntf@@QAAXW4SWIHW_TYPE_Power@@@Z 00102764 f   HWIntf.obj
 0001:00001890       ?WaitForSingleObjectReset@CHWIntf@@QAAKPAXK@Z 00102890 f   HWIntf.obj
 0001:000019ac       ?GetInternalPowerState@CHWIntf@@IAA?AW4ePowerInternalState@@XZ 001029ac f   HWIntf.obj
 0001:000019fc       ?SetInternalPowerState@CHWIntf@@IAAXW4ePowerInternalState@@@Z 001029fc f   HWIntf.obj
 0001:00001a48       ?GetModemPowerState@CHWIntf@@QAAJPAW4SWIHW_TYPE_Power@@@Z 00102a48 f   HWIntf.obj
 0001:00001c20       ?SetModemPower@CHWIntf@@QAAJW4SWIHW_TYPE_Power@@@Z 00102c20 f   HWIntf.obj
 0001:00002510       ?BlockingAutoSuspend@CHWIntf@@QAAJHPAX@Z 00103510 f   HWIntf.obj
 0001:000029f4       ??0CriticalSection@@QAA@XZ 001039f4 f i HWIntf.obj
 0001:00002a34       ??_GCriticalSection@@UAAPAXI@Z 00103a34 f i HWIntf.obj
 0001:00002a34       ??_ECriticalSection@@UAAPAXI@Z 00103a34 f i HWIntf.obj
 0001:00002a74       ??1CriticalSection@@UAA@XZ 00103a74 f i HWIntf.obj
 0001:00002aa0       ??_ECHWIntf@@UAAPAXI@Z     00103aa0 f i HWIntf.obj
 0001:00002aa0       ??_GCHWIntf@@UAAPAXI@Z     00103aa0 f i HWIntf.obj
 0001:00002ae0       ??0SWISYNCBLOCK@@QAA@PAVCriticalSection@@@Z 00103ae0 f i HWIntf.obj
 0001:00002b1c       ?Lock@CriticalSection@@QAA_NXZ 00103b1c f i HWIntf.obj
 0001:00002b4c       ??1SWISYNCBLOCK@@QAA@XZ    00103b4c f i HWIntf.obj
 0001:00002b68       ?Unlock@CriticalSection@@QAA_NXZ 00103b68 f i HWIntf.obj
 0001:00002b98       PulseEvent                 00103b98 f i HWIntf.obj
 0001:00002bcc       SetEvent                   00103bcc f i HWIntf.obj
 0001:00002c00       DllMain                    00103c00 f   SwiHWAux.obj
 0001:00002c84       SwiHWInitialize            00103c84 f   SwiHWAux.obj
 0001:00002d68       SwiHWUnInitialize          00103d68 f   SwiHWAux.obj
 0001:00002e3c       SwiHWSetPower              00103e3c f   SwiHWAux.obj
 0001:00002f64       SwiHWGetPower              00103f64 f   SwiHWAux.obj
 0001:00003010       SwiHWGetOEMIDStrA          00104010 f   SwiHWAux.obj
 0001:00003054       SwiHWRegisterCallback      00104054 f   SwiHWAux.obj
 0001:00003134       HWEnableAudio              00104134 f   SwiHWAux.obj
 0001:000031cc       HWGetAudioPath             001041cc f   SwiHWAux.obj
 0001:00003270       HWInitiateHostBoot         00104270 f   SwiHWAux.obj
 0001:00003308       HWSetVolumnLevel           00104308 f   SwiHWAux.obj
 0001:00003398       HWSetTetheredMode          00104398 f   SwiHWAux.obj
 0001:0000347c       ?PowerUpOperation@@YAXPAX@Z 0010447c f   SwiHWAux.obj
 0001:000034a4       HWSetDevicePowerState      001044a4 f   SwiHWAux.obj
 0001:00003718       ?WriteLog@@YAXKPBGZZ       00104718 f   sw_utilityG:sw_utilityG.dll
 0001:00003728       ?LogW@@YAXPBGZZ            00104728 f   sw_utilityG:sw_utilityG.dll
 0001:00003738       ?LogStoreFileLine@@YAXPAGH@Z 00104738 f   sw_utilityG:sw_utilityG.dll
 0001:00003748       ?SWAI_GetRegValue@@YAJPAUHKEY__@@PBG1AAK@Z 00104748 f   sw_utilityG:sw_utilityG.dll
 0001:00003758       ?LogC@@YAXPBGZZ            00104758 f   sw_utilityG:sw_utilityG.dll
 0001:00003768       ?SWAI_GetRegValue@@YAJPAUHKEY__@@PBG1PAGPAK@Z 00104768 f   sw_utilityG:sw_utilityG.dll
 0001:00003778       ?SetRegValue@@YAJPAUHKEY__@@PBG1K@Z 00104778 f   sw_utilityG:sw_utilityG.dll
 0001:00003788       ?GetRegValue@@YAJPAUHKEY__@@PBG1AAK@Z 00104788 f   sw_utilityG:sw_utilityG.dll
 0001:00003798       ??3@YAXPAX@Z               00104798 f   coredll:COREDLL.dll
 0001:000037a8       Sleep                      001047a8 f   coredll:COREDLL.dll
 0001:000037b8       GetProcAddressW            001047b8 f   coredll:COREDLL.dll
 0001:000037c8       LoadLibraryW               001047c8 f   coredll:COREDLL.dll
 0001:000037d8       wcscpy                     001047d8 f   coredll:COREDLL.dll
 0001:000037e8       memset                     001047e8 f   coredll:COREDLL.dll
 0001:000037f8       FreeLibrary                001047f8 f   coredll:COREDLL.dll
 0001:00003808       _snprintf                  00104808 f   coredll:COREDLL.dll
 0001:00003818       NKDbgPrintfW               00104818 f   coredll:COREDLL.dll
 0001:00003828       WaitForSingleObject        00104828 f   coredll:COREDLL.dll
 0001:00003838       DeleteCriticalSection      00104838 f   coredll:COREDLL.dll
 0001:00003848       free                       00104848 f   coredll:COREDLL.dll
 0001:00003858       RaiseException             00104858 f   coredll:COREDLL.dll
 0001:00003868       CreateEventW               00104868 f   coredll:COREDLL.dll
 0001:00003878       _purecall                  00104878 f   coredll:COREDLL.dll
 0001:00003888       InitializeCriticalSection  00104888 f   coredll:COREDLL.dll
 0001:00003898       CloseHandle                00104898 f   coredll:COREDLL.dll
 0001:000038a8       EnterCriticalSection       001048a8 f   coredll:COREDLL.dll
 0001:000038b8       LeaveCriticalSection       001048b8 f   coredll:COREDLL.dll
 0001:000038c8       WaitForMultipleObjects     001048c8 f   coredll:COREDLL.dll
 0001:000038d8       GetTickCount               001048d8 f   coredll:COREDLL.dll
 0001:000038e8       EventModify                001048e8 f   coredll:COREDLL.dll
 0001:000038f8       DisableThreadLibraryCalls  001048f8 f   coredll:COREDLL.dll
 0001:00003908       GetModuleFileNameW         00104908 f   coredll:COREDLL.dll
 0001:00003918       ??2@YAPAXI@Z               00104918 f   coredll:COREDLL.dll
 0001:00003928       CreateThread               00104928 f   coredll:COREDLL.dll
 0001:00003938       _DllMainCRTStartup         00104938 f   corelibc:pegdmain.obj
 0001:000039d0       __security_check_cookie    001049d0     corelibc:armsecgs.obj
 0001:000039e4       __gsfailure                001049e4     corelibc:armsecgs.obj
 0001:00003a28       _onexit                    00104a28 f   corelibc:onexit.obj
 0001:00003ad4       atexit                     00104ad4 f   corelibc:onexit.obj
 0001:00003af4       GetCurrentProcess          00104af4 f i corelibc:crt0dat.obj
 0001:00003afc       _cinit                     00104afc f   corelibc:crt0dat.obj
 0001:00003c6c       _exit                      00104c6c f   corelibc:crt0dat.obj
 0001:00003c84       _cexit                     00104c84 f   corelibc:crt0dat.obj
 0001:00003ca0       __security_init_cookie     00104ca0 f   corelibc:seccinit.obj
 0001:00003cf0       ?AtlAdvise@ATL@@YAJPAUIUnknown@@0ABU_GUID@@PAK@Z 00104cf0 f   atlsd:atlfuncs.obj
 0001:00003eac       ?AtlUnadvise@ATL@@YAJPAUIUnknown@@ABU_GUID@@K@Z 00104eac f   atlsd:atlfuncs.obj
 0001:00004064       ?AtlFreeMarshalStream@ATL@@YAJPAUIStream@@@Z 00105064 f   atlsd:atlfuncs.obj
 0001:0000411c       ?AtlMarshalPtrInProc@ATL@@YAJPAUIUnknown@@ABU_GUID@@PAPAUIStream@@@Z 0010511c f   atlsd:atlfuncs.obj
 0001:00004260       ?AtlUnmarshalPtr@ATL@@YAJPAUIStream@@ABU_GUID@@PAPAUIUnknown@@@Z 00105260 f   atlsd:atlfuncs.obj
 0001:00004380       ?AtlComModuleGetClassObject@ATL@@YAJPAU_ATL_COM_MODULE70@1@ABU_GUID@@1PAPAX@Z 00105380 f   atlsd:atlfuncs.obj
 0001:000046f8       ?AtlComModuleRegisterClassObjects@ATL@@YAJPAU_ATL_COM_MODULE70@1@KK@Z 001056f8 f   atlsd:atlfuncs.obj
 0001:00004818       ?AtlComModuleRevokeClassObjects@ATL@@YAJPAU_ATL_COM_MODULE70@1@@Z 00105818 f   atlsd:atlfuncs.obj
 0001:00004930       ?AtlWaitWithMessageLoop@ATL@@YAHPAX@Z 00105930 f   atlsd:atlfuncs.obj
 0001:00004ac8       ?AtlInternalQueryInterface@ATL@@YAJPAXPBU_ATL_INTMAP_ENTRY@1@ABU_GUID@@PAPAX@Z 00105ac8 f   atlsd:atlfuncs.obj
 0001:00004e50       ?AtlGetVersion@ATL@@YAKPAX@Z 00105e50 f   atlsd:atlfuncs.obj
 0001:00004e78       ?AtlWinModuleAddCreateWndData@ATL@@YAXPAU_ATL_WIN_MODULE70@1@PAU_AtlCreateWndData@1@PAX@Z 00105e78 f   atlsd:atlfuncs.obj
 0001:000050b4       ?AtlWinModuleExtractCreateWndData@ATL@@YAPAXPAU_ATL_WIN_MODULE70@1@@Z 001060b4 f   atlsd:atlfuncs.obj
 0001:00005300       ?AtlWinModuleInit@ATL@@YAJPAU_ATL_WIN_MODULE70@1@@Z 00106300 f   atlsd:atlfuncs.obj
 0001:00005450       ?AtlModuleAddTermFunc@ATL@@YAJPAU_ATL_MODULE70@1@P6AXK@ZK@Z 00106450 f   atlsd:atlfuncs.obj
 0001:0000565c       ?AtlCallTermFunc@ATL@@YAXPAU_ATL_MODULE70@1@@Z 0010665c f   atlsd:atlfuncs.obj
 0001:00005724       ??1?$CComPtr@UIConnectionPoint@@@ATL@@QAA@XZ 00106724 f i atlsd:atlfuncs.obj
 0001:00005724       ??1?$CComPtr@UIUnknown@@@ATL@@QAA@XZ 00106724 f i atlsd:atlbase.obj
 0001:00005724       ??1?$CComPtr@UIPersistStream@@@ATL@@QAA@XZ 00106724 f i atlsd:atlbase.obj
 0001:00005724       ??1?$CComPtr@UIConnectionPointContainer@@@ATL@@QAA@XZ 00106724 f i atlsd:atlfuncs.obj
 0001:0000574c       GetCurrentThreadId         0010674c f i atlsd:atlfuncs.obj
 0001:0000576c       ?IsWindowUnicode@ATL@@YAHPAUHWND__@@@Z 0010676c f i atlsd:atlfuncs.obj
 0001:00005794       ??1?$CComPtrBase@UIConnectionPointContainer@@@ATL@@QAA@XZ 00106794 f i atlsd:atlfuncs.obj
 0001:00005794       ??1?$CComPtrBase@UIConnectionPoint@@@ATL@@QAA@XZ 00106794 f i atlsd:atlfuncs.obj
 0001:00005794       ??1?$CComPtrBase@UIPersistStream@@@ATL@@QAA@XZ 00106794 f i atlsd:atlbase.obj
 0001:00005794       ??1?$CComPtrBase@UIUnknown@@@ATL@@QAA@XZ 00106794 f i atlsd:atlbase.obj
 0001:000057dc       ??I?$CComPtrBase@UIUnknown@@@ATL@@QAAPAPAUIUnknown@@XZ 001067dc f i atlsd:atlbase.obj
 0001:000057dc       ??I?$CComPtrBase@UIPersistStream@@@ATL@@QAAPAPAUIPersistStream@@XZ 001067dc f i atlsd:atlbase.obj
 0001:000057dc       ??I?$CComPtrBase@UIConnectionPointContainer@@@ATL@@QAAPAPAUIConnectionPointContainer@@XZ 001067dc f i atlsd:atlfuncs.obj
 0001:000057dc       ??I?$CComPtrBase@UIConnectionPoint@@@ATL@@QAAPAPAUIConnectionPoint@@XZ 001067dc f i atlsd:atlfuncs.obj
 0001:00005858       ??C?$CComPtrBase@UIConnectionPoint@@@ATL@@QBAPAV?$_NoAddRefReleaseOnCComPtr@UIConnectionPoint@@@1@XZ 00106858 f i atlsd:atlfuncs.obj
 0001:00005858       ??C?$CComPtrBase@UIPersistStream@@@ATL@@QBAPAV?$_NoAddRefReleaseOnCComPtr@UIPersistStream@@@1@XZ 00106858 f i atlsd:atlbase.obj
 0001:00005858       ??C?$CComPtrBase@UIConnectionPointContainer@@@ATL@@QBAPAV?$_NoAddRefReleaseOnCComPtr@UIConnectionPointContainer@@@1@XZ 00106858 f i atlsd:atlfuncs.obj
 0001:00005858       ??C?$CComPtrBase@UIUnknown@@@ATL@@QBAPAV?$_NoAddRefReleaseOnCComPtr@UIUnknown@@@1@XZ 00106858 f i atlsd:atlbase.obj
 0001:000058d8       ??0?$CComPtrBase@UIConnectionPointContainer@@@ATL@@IAA@XZ 001068d8 f i atlsd:atlfuncs.obj
 0001:000058d8       ??0?$CComPtrBase@UIUnknown@@@ATL@@IAA@XZ 001068d8 f i atlsd:atlbase.obj
 0001:000058d8       ??0?$CComPtrBase@UIConnectionPoint@@@ATL@@IAA@XZ 001068d8 f i atlsd:atlfuncs.obj
 0001:000058d8       ??0?$CComPtrBase@UIPersistStream@@@ATL@@IAA@XZ 001068d8 f i atlsd:atlbase.obj
 0001:0000590c       ?InlineIsEqualGUID@ATL@@YAHABU_GUID@@0@Z 0010690c f i atlsd:atlfuncs.obj
 0001:000059c0       ??0CTraceFileAndLineInfo@ATL@@QAA@PBDH@Z 001069c0 f i atlsd:atlfuncs.obj
 0001:00005a04       ??RCTraceFileAndLineInfo@ATL@@QBAXKIPB_WZZ 00106a04 f i atlsd:atlfuncs.obj
 0001:00005a7c       ?TraceV@CTrace@ATL@@QBAXPBDHKIPB_WPAD@Z 00106a7c f i atlsd:atlfuncs.obj
 0001:00005ad8       ??BCTraceCategory@ATL@@QBAKXZ 00106ad8 f i atlsd:atlfuncs.obj
 0001:00005b0c       ?Init@CComCriticalSection@ATL@@QAAJXZ 00106b0c f i atlsd:atlfuncs.obj
 0001:00005bb0       ?RevokeClassObject@_ATL_OBJMAP_ENTRY30@ATL@@QAAJXZ 00106bb0 f i atlsd:atlfuncs.obj
 0001:00005c18       ?RegisterClassObject@_ATL_OBJMAP_ENTRY30@ATL@@QAAJKK@Z 00106c18 f i atlsd:atlfuncs.obj
 0001:00005d10       ?InlineIsEqualUnknown@ATL@@YAHABU_GUID@@@Z 00106d10 f i atlsd:atlfuncs.obj
 0001:00005d98       ??0?$CComCritSecLock@VCComCriticalSection@ATL@@@ATL@@QAA@AAVCComCriticalSection@1@_N@Z 00106d98 f i atlsd:atlfuncs.obj
 0001:00005e28       ?AtlThrowImpl@ATL@@YAXJ@Z  00106e28 f i atlsd:atlfuncs.obj
 0001:00005f38       ??1?$CComCritSecLock@VCComCriticalSection@ATL@@@ATL@@QAA@XZ 00106f38 f i atlsd:atlfuncs.obj
 0001:00005f74       ?Unlock@?$CComCritSecLock@VCComCriticalSection@ATL@@@ATL@@QAAXXZ 00106f74 f i atlsd:atlfuncs.obj
 0001:00006014       ?Unlock@CComCriticalSection@ATL@@QAAJXZ 00107014 f i atlsd:atlfuncs.obj
 0001:00006050       ?Lock@?$CComCritSecLock@VCComCriticalSection@ATL@@@ATL@@QAAJXZ 00107050 f i atlsd:atlfuncs.obj
 0001:00006120       ?Lock@CComCriticalSection@ATL@@QAAJXZ 00107120 f i atlsd:atlfuncs.obj
 0001:0000615c       AtlRawDllMain              0010715c f   atlsd:atlbase.obj
 0001:0000625c       ?CoDisconnectObject@ATL@@YAJPAUIUnknown@@K@Z 0010725c f   atlsd:atlbase.obj
 0001:000063b0       ?CoInitialize@ATL@@YAJPAX@Z 001073b0 f   atlsd:atlbase.obj
 0001:00006464       ?CoRevokeClassObject@ATL@@YAJK@Z 00107464 f   atlsd:atlbase.obj
 0001:00006518       ?CoRegisterClassObject@ATL@@YAJABU_GUID@@PAUIUnknown@@KKPAK@Z 00107518 f   atlsd:atlbase.obj
 0001:000065e0       ?CoMarshalInterface@ATL@@YAJPAUIStream@@ABU_GUID@@PAUIUnknown@@KPAXK@Z 001075e0 f   atlsd:atlbase.obj
 0001:000066b0       ?CoUnmarshalInterface@ATL@@YAJPAUIStream@@ABU_GUID@@PAPAX@Z 001076b0 f   atlsd:atlbase.obj
 0001:0000676c       ?CoReleaseMarshalData@ATL@@YAJPAUIStream@@@Z 0010776c f   atlsd:atlbase.obj
 0001:00006820       ?OleSaveToStream@ATL@@YAJPAUIPersistStream@@PAUIStream@@@Z 00107820 f   atlsd:atlbase.obj
 0001:000069d8       ?OleLoadFromStream@ATL@@YAJPAUIStream@@ABU_GUID@@PAPAX@Z 001079d8 f   atlsd:atlbase.obj
 0001:00006d04       ??0CAtlBaseModule@ATL@@QAA@XZ 00107d04 f   atlsd:atlbase.obj
 0001:00006e90       ??1CAtlBaseModule@ATL@@QAA@XZ 00107e90 f   atlsd:atlbase.obj
 0001:00006ed0       ?AddResourceInstance@CAtlBaseModule@ATL@@QAA_NPAUHINSTANCE__@@@Z 00107ed0 f   atlsd:atlbase.obj
 0001:0000706c       ?RemoveResourceInstance@CAtlBaseModule@ATL@@QAA_NPAUHINSTANCE__@@@Z 0010806c f   atlsd:atlbase.obj
 0001:00007280       ?GetHInstanceAt@CAtlBaseModule@ATL@@QAAPAUHINSTANCE__@@H@Z 00108280 f   atlsd:atlbase.obj
 0001:000074b4       ??0_ATL_BASE_MODULE70@ATL@@QAA@XZ 001084b4 f i atlsd:atlbase.obj
 0001:00007514       ??1_ATL_BASE_MODULE70@ATL@@QAA@XZ 00108514 f i atlsd:atlbase.obj
 0001:00007558       ?_AtlGetThisModuleHandle@ATL@@YAPAUHINSTANCE__@@XZ 00108558 f i atlsd:atlbase.obj
 0001:000075b8       ?Add@?$CSimpleArray@PAUHINSTANCE__@@V?$CSimpleArrayEqualHelper@PAUHINSTANCE__@@@ATL@@@ATL@@QAAHABQAUHINSTANCE__@@@Z 001085b8 f i atlsd:atlbase.obj
 0001:000075b8       ?Add@?$CSimpleArray@KV?$CSimpleArrayEqualHelper@K@ATL@@@ATL@@QAAHABK@Z 001085b8 f i atlsd:Allocate.obj
 0001:00007708       ?RemoveAt@?$CSimpleArray@KV?$CSimpleArrayEqualHelper@K@ATL@@@ATL@@QAAHH@Z 00108708 f i atlsd:Allocate.obj
 0001:00007708       ?RemoveAt@?$CSimpleArray@PAUHINSTANCE__@@V?$CSimpleArrayEqualHelper@PAUHINSTANCE__@@@ATL@@@ATL@@QAAHH@Z 00108708 f i atlsd:atlbase.obj
 0001:00007880       ??A?$CSimpleArray@KV?$CSimpleArrayEqualHelper@K@ATL@@@ATL@@QAAAAKH@Z 00108880 f i atlsd:Allocate.obj
 0001:00007880       ??A?$CSimpleArray@PAUHINSTANCE__@@V?$CSimpleArrayEqualHelper@PAUHINSTANCE__@@@ATL@@@ATL@@QAAAAPAUHINSTANCE__@@H@Z 00108880 f i atlsd:atlbase.obj
 0001:00007964       ??0Wrapper@?$CSimpleArray@PAUHINSTANCE__@@V?$CSimpleArrayEqualHelper@PAUHINSTANCE__@@@ATL@@@ATL@@QAA@ABQAUHINSTANCE__@@@Z 00108964 f i atlsd:atlbase.obj
 0001:00007964       ??0Wrapper@?$CSimpleArray@KV?$CSimpleArrayEqualHelper@K@ATL@@@ATL@@QAA@ABK@Z 00108964 f i atlsd:Allocate.obj
 0001:0000799c       ?memmove_s@Checked@ATL@@YAXPAXIPBXI@Z 0010899c f i atlsd:atlbase.obj
 0001:000079f0       ?AtlCrtErrorCheck@ATL@@YAHH@Z 001089f0 f i atlsd:atlbase.obj
 0001:00007abc       ??0?$CComPtr@UIPersistStream@@@ATL@@QAA@XZ 00108abc f i atlsd:atlbase.obj
 0001:00007abc       ??0?$CComPtr@UIConnectionPoint@@@ATL@@QAA@XZ 00108abc f i atlsd:atlfuncs.obj
 0001:00007abc       ??0?$CComPtr@UIConnectionPointContainer@@@ATL@@QAA@XZ 00108abc f i atlsd:atlfuncs.obj
 0001:00007abc       ??0?$CComPtr@UIUnknown@@@ATL@@QAA@XZ 00108abc f i atlsd:atlbase.obj
 0001:00007afc       ??0CTraceCategory@ATL@@QAA@PB_WI@Z 00108afc f i atlsd:atltrace.obj
 0001:00007b80       ?ChangeCategory@CTrace@ATL@@QAA_NKIW4ATLTRACESTATUS@2@@Z 00108b80 f i atlsd:atltrace.obj
 0001:00007bf0       ?RegisterCategory@CTrace@ATL@@QAAKPB_W@Z 00108bf0 f i atlsd:atltrace.obj
 0001:00007c3c       ??0CAtlAllocator@@QAA@XZ   00108c3c f i atlsd:Externs.obj
 0001:00007ccc       ??0CTraceSnapshot@@QAA@XZ  00108ccc f i atlsd:Externs.obj
 0001:00007d28       ??0?$CSimpleArray@UCModuleInfo@CTraceSnapshot@@V?$CSimpleArrayEqualHelper@UCModuleInfo@CTraceSnapshot@@@ATL@@@ATL@@QAA@XZ 00108d28 f i atlsd:Externs.obj
 0001:00007d28       ??0?$CSimpleArray@KV?$CSimpleArrayEqualHelper@K@ATL@@@ATL@@QAA@XZ 00108d28 f i atlsd:Externs.obj
 0001:00007d28       ??0?$CSimpleArray@PAUHINSTANCE__@@V?$CSimpleArrayEqualHelper@PAUHINSTANCE__@@@ATL@@@ATL@@QAA@XZ 00108d28 f i atlsd:atlbase.obj
 0001:00007eec       GetCurrentProcessId        00108eec f i atlsd:Externs.obj
 0001:00007f0c       ??0CAtlException@ATL@@QAA@J@Z 00108f0c f i atlsd:Externs.obj
 0001:00007f40       ??0CTrace@ATL@@AAA@P6AHHPB_WH00ZZ@Z 00108f40 f i atlsd:Externs.obj
 0001:00007fc8       ??1CAtlAllocator@@QAA@XZ   00108fc8 f i atlsd:Externs.obj
 0001:00008008       ??1CTraceSnapshot@@QAA@XZ  00109008 f i atlsd:Externs.obj
 0001:00008048       ??1?$CSimpleArray@KV?$CSimpleArrayEqualHelper@K@ATL@@@ATL@@QAA@XZ 00109048 f i atlsd:Externs.obj
 0001:00008048       ??1?$CSimpleArray@PAUHINSTANCE__@@V?$CSimpleArrayEqualHelper@PAUHINSTANCE__@@@ATL@@@ATL@@QAA@XZ 00109048 f i atlsd:atlbase.obj
 0001:00008048       ??1?$CSimpleArray@UCModuleInfo@CTraceSnapshot@@V?$CSimpleArrayEqualHelper@UCModuleInfo@CTraceSnapshot@@@ATL@@@ATL@@QAA@XZ 00109048 f i atlsd:Externs.obj
 0001:00008070       ?RemoveAll@?$CSimpleArray@KV?$CSimpleArrayEqualHelper@K@ATL@@@ATL@@QAAXXZ 00109070 f i atlsd:Externs.obj
 0001:00008070       ?RemoveAll@?$CSimpleArray@PAUHINSTANCE__@@V?$CSimpleArrayEqualHelper@PAUHINSTANCE__@@@ATL@@@ATL@@QAAXXZ 00109070 f i atlsd:atlbase.obj
 0001:00008070       ?RemoveAll@?$CSimpleArray@UCModuleInfo@CTraceSnapshot@@V?$CSimpleArrayEqualHelper@UCModuleInfo@CTraceSnapshot@@@ATL@@@ATL@@QAAXXZ 00109070 f i atlsd:Externs.obj
 0001:00008114       ??1CTrace@ATL@@AAA@XZ      00109114 f i atlsd:Externs.obj
 0001:00008144       ?NotifyTool@ATL@@YAXXZ     00109144 f   atlsd:AtlDebugAPI.obj
 0001:000081bc       AtlTraceRegister           001091bc f   atlsd:AtlDebugAPI.obj
 0001:000082b8       AtlTraceUnregister         001092b8 f   atlsd:AtlDebugAPI.obj
 0001:00008318       AtlTraceRegisterCategoryU  00109318 f   atlsd:AtlDebugAPI.obj
 0001:000083a4       AtlTraceModifyProcess      001093a4 f   atlsd:AtlDebugAPI.obj
 0001:00008524       AtlTraceModifyModule       00109524 f   atlsd:AtlDebugAPI.obj
 0001:000086c4       AtlTraceModifyCategory     001096c4 f   atlsd:AtlDebugAPI.obj
 0001:00008804       AtlTraceGetProcess         00109804 f   atlsd:AtlDebugAPI.obj
 0001:000089a4       AtlTraceGetModule          001099a4 f   atlsd:AtlDebugAPI.obj
 0001:00008b94       AtlTraceGetCategory        00109b94 f   atlsd:AtlDebugAPI.obj
 0001:00008d38       AtlTraceGetUpdateEventNameU 00109d38 f   atlsd:AtlDebugAPI.obj
 0001:00008d8c       AtlTraceGetUpdateEventNameU_s 00109d8c f   atlsd:AtlDebugAPI.obj
 0001:00008de4       AtlTraceVU                 00109de4 f   atlsd:AtlDebugAPI.obj
 0001:000090f4       AtlTraceOpenProcess        0010a0f4 f   atlsd:AtlDebugAPI.obj
 0001:00009150       AtlTraceCloseProcess       0010a150 f   atlsd:AtlDebugAPI.obj
 0001:0000928c       AtlTraceSnapshotProcess    0010a28c f   atlsd:AtlDebugAPI.obj
 0001:00009364       AtlTraceGetProcessInfo     0010a364 f   atlsd:AtlDebugAPI.obj
 0001:00009694       AtlTraceGetModuleInfo      0010a694 f   atlsd:AtlDebugAPI.obj
 0001:00009988       AtlTraceGetCategoryInfo    0010a988 f   atlsd:AtlDebugAPI.obj
 0001:0000a040       ?GetProcess@CAtlAllocator@@QBAPAVCAtlTraceProcess@@XZ 0010b040 f i atlsd:AtlDebugAPI.obj
 0001:0000a070       ?Name@CAtlTraceCategory@@QBAPB_WXZ 0010b070 f i atlsd:AtlDebugAPI.obj
 0001:0000a09c       ?Path@CAtlTraceModuleInfo@@QBAPB_WXZ 0010b09c f i atlsd:AtlDebugAPI.obj
 0001:0000a0c8       ?Name@CAtlTraceModuleInfo@@QBAPB_WXZ 0010b0c8 f i atlsd:AtlDebugAPI.obj
 0001:0000a0f4       ?Id@CAtlTraceProcess@@QBAKXZ 0010b0f4 f i atlsd:AtlDebugAPI.obj
 0001:0000a128       ?CrtDbgReport@CAtlTraceModule@@QBAP6AHHPB_WH00ZZXZ 0010b128 f i atlsd:AtlDebugAPI.obj
 0001:0000a15c       ??A?$CSimpleArray@UCModuleInfo@CTraceSnapshot@@V?$CSimpleArrayEqualHelper@UCModuleInfo@CTraceSnapshot@@@ATL@@@ATL@@QAAAAUCModuleInfo@CTraceSnapshot@@H@Z 0010b15c f i atlsd:AtlDebugAPI.obj
 0001:0000a240       ?wcscpy_s@Checked@ATL@@YAXPA_WIPB_W@Z 0010b240 f i atlsd:AtlDebugAPI.obj
 0001:0000a298       ?Init@CAtlAllocator@@QAA_NPB_WK@Z 0010b298 f   atlsd:Allocate.obj
 0001:0000a770       ?Close@CAtlAllocator@@QAAX_N@Z 0010b770 f   atlsd:Allocate.obj
 0001:0000a840       ?GetModule@CAtlAllocator@@QBAPAVCAtlTraceModule@@H@Z 0010b840 f   atlsd:Allocate.obj
 0001:0000a954       ?GetCategory@CAtlAllocator@@QBAPAVCAtlTraceCategory@@H@Z 0010b954 f   atlsd:Allocate.obj
 0001:0000aa9c       ?GetCategoryCount@CAtlAllocator@@QBAHH@Z 0010ba9c f   atlsd:Allocate.obj
 0001:0000ab74       ?GetCategoryCount@CAtlAllocator@@QBAHABVCAtlTraceModule@@@Z 0010bb74 f   atlsd:Allocate.obj
 0001:0000ac10       ?GetModuleCount@CAtlAllocator@@QBAHXZ 0010bc10 f   atlsd:Allocate.obj
 0001:0000acb0       ?FindModule@CAtlAllocator@@QBA_NPB_WPAI@Z 0010bcb0 f   atlsd:Allocate.obj
 0001:0000ada4       ?AddModule@CAtlAllocator@@QAAHPAUHINSTANCE__@@@Z 0010bda4 f   atlsd:Allocate.obj
 0001:0000b0ec       ?AddCategory@CAtlAllocator@@QAAHHPB_W@Z 0010c0ec f   atlsd:Allocate.obj
 0001:0000b4f4       ?RemoveModule@CAtlAllocator@@QAA_NH@Z 0010c4f4 f   atlsd:Allocate.obj
 0001:0000b628       ?CleanUp@CAtlAllocator@@QAAXXZ 0010c628 f   atlsd:Allocate.obj
 0001:0000b654       ?TakeSnapshot@CAtlAllocator@@QAAXXZ 0010c654 f   atlsd:Allocate.obj
 0001:0000b990       ?ReleaseSnapshot@CAtlAllocator@@QAAXXZ 0010c990 f   atlsd:Allocate.obj
 0001:0000bb30       ?IncRef@CAtlTraceProcess@@QAAIXZ 0010cb30 f i atlsd:Allocate.obj
 0001:0000bb88       ?Base@CAtlTraceProcess@@QBAPAXXZ 0010cb88 f i atlsd:Allocate.obj
 0001:0000bbbc       ?DecRef@CAtlTraceProcess@@QAAIXZ 0010cbbc f i atlsd:Allocate.obj
 0001:0000bc14       ?ModuleCount@CAtlTraceProcess@@QBAHXZ 0010cc14 f i atlsd:Allocate.obj
 0001:0000bc48       ?MaxSize@CAtlTraceProcess@@QBAKXZ 0010cc48 f i atlsd:Allocate.obj
 0001:0000bc78       ?CategoryCount@CAtlTraceProcess@@QBAHXZ 0010cc78 f i atlsd:Allocate.obj
 0001:0000bca8       ?TryAllocate@CAtlTraceSettings@@QAA_NXZ 0010cca8 f i atlsd:Allocate.obj
 0001:0000bd2c       ?MarkValid@CAtlTraceSettings@@QAAXJ@Z 0010cd2c f i atlsd:Allocate.obj
 0001:0000bda8       ?IncModuleCount@CAtlTraceProcess@@QAAXI@Z 0010cda8 f i atlsd:Allocate.obj
 0001:0000bde4       ?TryAddRef@CAtlTraceSettings@@QAA_NXZ 0010cde4 f i atlsd:Allocate.obj
 0001:0000be74       ?Release@CAtlTraceSettings@@QAAXXZ 0010ce74 f i atlsd:Allocate.obj
 0001:0000bed0       ?IncCategoryCount@CAtlTraceProcess@@QAAXI@Z 0010ced0 f i atlsd:Allocate.obj
 0001:0000bf04       ?Add@?$CSimpleArray@UCModuleInfo@CTraceSnapshot@@V?$CSimpleArrayEqualHelper@UCModuleInfo@CTraceSnapshot@@@ATL@@@ATL@@QAAHABUCModuleInfo@CTraceSnapshot@@@Z 0010cf04 f i atlsd:Allocate.obj
 0001:0000c05c       ?GetSize@?$CSimpleArray@PAUHINSTANCE__@@V?$CSimpleArrayEqualHelper@PAUHINSTANCE__@@@ATL@@@ATL@@QBAHXZ 0010d05c f i atlsd:atlbase.obj
 0001:0000c05c       ?GetSize@?$CSimpleArray@UCModuleInfo@CTraceSnapshot@@V?$CSimpleArrayEqualHelper@UCModuleInfo@CTraceSnapshot@@@ATL@@@ATL@@QBAHXZ 0010d05c f i atlsd:AtlDebugAPI.obj
 0001:0000c05c       ?GetSize@?$CSimpleArray@KV?$CSimpleArrayEqualHelper@K@ATL@@@ATL@@QBAHXZ 0010d05c f i atlsd:Allocate.obj
 0001:0000c08c       ?InternalSetAtIndex@?$CSimpleArray@UCModuleInfo@CTraceSnapshot@@V?$CSimpleArrayEqualHelper@UCModuleInfo@CTraceSnapshot@@@ATL@@@ATL@@QAAXHABUCModuleInfo@CTraceSnapshot@@@Z 0010d08c f i atlsd:Allocate.obj
 0001:0000c11c       ?InternalSetAtIndex@?$CSimpleArray@KV?$CSimpleArrayEqualHelper@K@ATL@@@ATL@@QAAXHABK@Z 0010d11c f i atlsd:Allocate.obj
 0001:0000c11c       ?InternalSetAtIndex@?$CSimpleArray@PAUHINSTANCE__@@V?$CSimpleArrayEqualHelper@PAUHINSTANCE__@@@ATL@@@ATL@@QAAXHABQAUHINSTANCE__@@@Z 0010d11c f i atlsd:atlbase.obj
 0001:0000c1ac       ??0Wrapper@?$CSimpleArray@UCModuleInfo@CTraceSnapshot@@V?$CSimpleArrayEqualHelper@UCModuleInfo@CTraceSnapshot@@@ATL@@@ATL@@QAA@ABUCModuleInfo@CTraceSnapshot@@@Z 0010d1ac f i atlsd:Allocate.obj
 0001:0000c1e4       ??$?2PAUHINSTANCE__@@@Wrapper@?$CSimpleArray@PAUHINSTANCE__@@V?$CSimpleArrayEqualHelper@PAUHINSTANCE__@@@ATL@@@ATL@@SAPAXIPAPAUHINSTANCE__@@@Z 0010d1e4 f i atlsd:atlbase.obj
 0001:0000c1e4       ??2@YAPAXIPAX@Z            0010d1e4 f i atlsd:Allocate.obj
 0001:0000c1e4       ??$?2K@Wrapper@?$CSimpleArray@KV?$CSimpleArrayEqualHelper@K@ATL@@@ATL@@SAPAXIPAK@Z 0010d1e4 f i atlsd:Allocate.obj
 0001:0000c1e4       ??$?2UCModuleInfo@CTraceSnapshot@@@Wrapper@?$CSimpleArray@UCModuleInfo@CTraceSnapshot@@V?$CSimpleArrayEqualHelper@UCModuleInfo@CTraceSnapshot@@@ATL@@@ATL@@SAPAXIPAUCModuleInfo@CTraceSnapshot@@@Z 0010d1e4 f i atlsd:Allocate.obj
 0001:0000c20c       ??0CAtlTraceModuleInfo@@QAA@XZ 0010d20c f   atlsd:AtlTraceModuleManager.obj
 0001:0000c280       ?Reset@CAtlTraceModuleInfo@@QAAXPAUHINSTANCE__@@@Z 0010d280 f   atlsd:AtlTraceModuleManager.obj
 0001:0000c41c       ??0CAtlTraceCategory@@QAA@XZ 0010d41c f   atlsd:AtlTraceModuleManager.obj
 0001:0000c488       ?Reset@CAtlTraceCategory@@QAAXPB_WJ@Z 0010d488 f   atlsd:AtlTraceModuleManager.obj
 0001:0000c508       ??0CAtlTraceModule@@QAA@XZ 0010d508 f   atlsd:AtlTraceModuleManager.obj
 0001:0000c574       ?CrtDbgReport@CAtlTraceModule@@QAAXP6AHHPB_WH00ZZ@Z 0010d574 f   atlsd:AtlTraceModuleManager.obj
 0001:0000c5c8       ??0CAtlTraceProcess@@QAA@K@Z 0010d5c8 f   atlsd:AtlTraceModuleManager.obj
 0001:0000c740       ?GetNextCookie@CAtlTraceProcess@@QAAJXZ 0010d740 f   atlsd:AtlTraceModuleManager.obj
 0001:0000c788       ??0CAtlTraceSettings@@QAA@XZ 0010d788 f i atlsd:AtlTraceModuleManager.obj
 0001:0000c7ec       __InternalCxxFrameHandler  0010d7ec f   LIBCMTD:frame_ce.obj
 0001:0000c9c8       __CxxFrameHandler3         0010d9c8 f   LIBCMTD:frame_ce.obj
 0001:0000d1a4       __FrameUnwindToState       0010e1a4 f   LIBCMTD:frame_ce.obj
 0001:0000df50       ?_DestructExceptionObject@@YAXPAUEHExceptionRecord@@E@Z 0010ef50 f   LIBCMTD:frame_ce.obj
 0001:0000e0a0       ?_OffsetToAddress@@YAPAXHPAKK@Z 0010f0a0 f   LIBCMTD:frame_ce.obj
 0001:0000e12c       ?FindFrameInfo@@YAPAU_FrameInfo@@PAK@Z 0010f12c f   LIBCMTD:frame_ce.obj
 0001:0000e1b4       ?FindCatchFrameInfo@@YAPAU_FrameInfo@@PAK@Z 0010f1b4 f   LIBCMTD:frame_ce.obj
 0001:0000e238       ?_GetRangeOfTrysToCheck@@YAPBU_s_TryBlockMapEntry@@PBU_s_FuncInfo@@HHPAI1@Z 0010f238 f   LIBCMTD:frame_ce.obj
 0001:0000e330       __GSHandlerCheckCommon     0010f330 f   LIBCMTD:gshandler.obj
 0001:0000e378       __GSHandlerCheck           0010f378 f   LIBCMTD:gshandler.obj
 0001:0000e3a8       _CrtDbgReportW             0010f3a8 f   LIBCMTD:dbgrpt.obj
 0001:0000e420       _CrtDbgReportTV            0010f420 f i LIBCMTD:dbgrpt.obj
 0001:0000e47c       __crtMessageWindowW        0010f47c f   LIBCMTD:dbgrpt.obj
 0001:0000eb54       _invoke_watson_if_error    0010fb54 f i LIBCMTD:dbgrpt.obj
 0001:0000eba8       memmove_s                  0010fba8 f   LIBCMTD:memmove_s.obj
 0001:0000ee1c       wcscpy_s                   0010fe1c f   LIBCMTD:wcscpy_s.obj
 0001:0000f290       wcsncpy_s                  00110290 f   LIBCMTD:wcsncpy_s.obj
 0001:0000f890       GetCRTStorage              00110890 f   LIBCMTD:corecrt.obj
 0001:0000f9a0       TlsAlloc                   001109a0 f i LIBCMTD:corecrt.obj
 0001:0000f9dc       TlsFree                    001109dc f i LIBCMTD:corecrt.obj
 0001:0000fa20       ?FindFrameForUnwind@@YAPAKPAKPBU_s_FuncInfo@@@Z 00110a20 f   LIBCMTD:mdframe_arm.obj
 0001:0000fab8       ?FindCatchFrame@@YAPAKPAKK@Z 00110ab8 f   LIBCMTD:mdframe_arm.obj
 0001:0000fb50       ?AdjustFrameForCatch@@YAPAKPAKPBU_s_FuncInfo@@@Z 00110b50 f   LIBCMTD:mdframe_arm.obj
 0001:0000fbf0       ?GetCurrentState@@YAHPAKPAU_DISPATCHER_CONTEXT@@PBU_s_FuncInfo@@@Z 00110bf0 f   LIBCMTD:ehstate_arm_mips.obj
 0001:0000fccc       _CallSettingFrame          00110ccc     LIBCMTD:handlers_arm.obj
 0001:0000fd10       _mtinitlocks               00110d10 f   LIBCMTD:mlock.obj
 0001:0000fe30       _mtinitlocknum             00110e30 f   LIBCMTD:mlock.obj
 0001:0000ff98       _lock                      00110f98 f   LIBCMTD:mlock.obj
 0001:00010094       _unlock                    00111094 f   LIBCMTD:mlock.obj
 0001:000100d4       _lockerr_exit              001110d4 f   LIBCMTD:mlock.obj
 0001:000100fc       _CrtDbgBreak               001110fc f   LIBCMTD:dbgrptt.obj
 0001:0001010c       _VCrtDbgReportW            0011110c f   LIBCMTD:dbgrptt.obj
 0001:00010cc4       _invalid_parameter         00111cc4 f   LIBCMTD:invarginternal.obj
 0001:00010d08       __crtMessageBoxW           00111d08 f   LIBCMTD:crtmbox.obj
 0001:00010f6c       _invoke_watson             00111f6c f   LIBCMTD:invarg.obj
 0001:00010fa8       __crtInitCritSecAndSpinCount 00111fa8 f   LIBCMTD:initcrit.obj
 0001:000110d8       _amsg_exit                 001120d8 f   LIBCMTD:crt0dat.obj
 0001:00011104       __crtExitProcess           00112104 f   LIBCMTD:crt0dat.obj
 0001:0001114c       strcpy_s                   0011214c f   LIBCMTD:strcpy_s.obj
 0001:000115a0       wcscat_s                   001125a0 f   LIBCMTD:wcscat_s.obj
 0001:00011b84       _itow_s                    00112b84 f   LIBCMTD:xtows.obj
 0001:00012210       _decode_pointer            00113210 f   LIBCMTD:tidtable.obj
 0001:00012210       _encode_pointer            00113210 f   LIBCMTD:tidtable.obj
 0001:00012238       _encoded_null              00113238 f   LIBCMTD:tidtable.obj
 0001:00012270       __report_gsfailure         00113270 f   coredll:COREDLL.dll
 0001:00012280       LocalReAlloc               00113280 f   coredll:COREDLL.dll
 0001:00012290       LocalAlloc                 00113290 f   coredll:COREDLL.dll
 0001:000122a0       LocalSize                  001132a0 f   coredll:COREDLL.dll
 0001:000122b0       LocalFree                  001132b0 f   coredll:COREDLL.dll
 0001:000122c0       __security_gen_cookie      001132c0 f   coredll:COREDLL.dll
 0001:000122d0       DispatchMessageW           001132d0 f   coredll:COREDLL.dll
 0001:000122e0       TranslateMessage           001132e0 f   coredll:COREDLL.dll
 0001:000122f0       GetMessageW                001132f0 f   coredll:COREDLL.dll
 0001:00012300       PeekMessageW               00113300 f   coredll:COREDLL.dll
 0001:00012310       MsgWaitForMultipleObjectsEx 00113310 f   coredll:COREDLL.dll
 0001:00012320       __C_specific_handler       00113320 f   coredll:COREDLL.dll
 0001:00012330       GetModuleHandleW           00113330 f   coredll:COREDLL.dll
 0001:00012340       realloc                    00113340 f   coredll:COREDLL.dll
 0001:00012350       _snwprintf                 00113350 f   coredll:COREDLL.dll
 0001:00012360       memcpy                     00113360 f   coredll:COREDLL.dll
 0001:00012370       __CxxThrowException        00113370 f   coredll:COREDLL.dll
 0001:00012380       ??_7type_info@@6B@         00113380 f   coredll:COREDLL.dll
 0001:00012390       OpenEventW                 00113390 f   coredll:COREDLL.dll
 0001:000123a0       OutputDebugStringW         001133a0 f   coredll:COREDLL.dll
 0001:000123b0       _vsnwprintf                001133b0 f   coredll:COREDLL.dll
 0001:000123c0       VirtualAlloc               001133c0 f   coredll:COREDLL.dll
 0001:000123d0       UnmapViewOfFile            001133d0 f   coredll:COREDLL.dll
 0001:000123e0       memcmp                     001133e0 f   coredll:COREDLL.dll
 0001:000123f0       GetSystemInfo              001133f0 f   coredll:COREDLL.dll
 0001:00012400       MapViewOfFile              00113400 f   coredll:COREDLL.dll
 0001:00012410       GetLastError               00113410 f   coredll:COREDLL.dll
 0001:00012420       CreateFileMappingW         00113420 f   coredll:COREDLL.dll
 0001:00012430       _wcsicmp                   00113430 f   coredll:COREDLL.dll
 0001:00012440       InterlockedIncrement       00113440 f   coredll:COREDLL.dll
 0001:00012450       InterlockedDecrement       00113450 f   coredll:COREDLL.dll
 0001:00012460       wcslen                     00113460 f   coredll:COREDLL.dll
 0001:00012470       strcmp                     00113470 f   coredll:COREDLL.dll
 0001:00012480       ?terminate@std@@YAXXZ      00113480 f   coredll:COREDLL.dll
 0001:00012490       memmove                    00113490 f   coredll:COREDLL.dll
 0001:000124a0       malloc                     001134a0 f   coredll:COREDLL.dll
 0001:000124b0       TlsSetValue                001134b0 f   coredll:COREDLL.dll
 0001:000124c0       TlsGetValue                001134c0 f   coredll:COREDLL.dll
 0001:000124d0       InterlockedCompareExchange 001134d0 f   coredll:COREDLL.dll
 0001:000124e0       TlsCall                    001134e0 f   coredll:COREDLL.dll
 0001:000124f0       WriteFile                  001134f0 f   coredll:COREDLL.dll
 0001:00012500       wcstombs                   00113500 f   coredll:COREDLL.dll
 0001:00012510       SetLastError               00113510 f   coredll:COREDLL.dll
 0001:00012520       TerminateProcess           00113520 f   coredll:COREDLL.dll
 0001:00012530       CreateStreamOnHGlobal      00113530 f   ole32:ole32.dll
 0001:00012540       WriteClassStm              00113540 f   ole32:ole32.dll
 0001:00012550       CoCreateInstance           00113550 f   ole32:ole32.dll
 0001:00012560       ReadClassStm               00113560 f   ole32:ole32.dll
 0002:00001a20       ??_7CCEHWIntf@@6B@         00115a20     CEHWIntf.obj
 0002:00001a48       ??_C@_1EA@JHMKKLFC@?$AAn?$AAI?$AAn?$AAd?$AAe?$AAx?$AA?5?$AA?$DO?$AA?$DN?$AA?5?$AA0?$AA?5?$AA?$CG?$AA?$CG?$AA?5?$AAn?$AAI?$AAn?$AAd?$AAe?$AAx?$AA?5?$AA?$DM?$AA?5?$AAm?$AA_?$AAn?$AAS?$AAi?$AAz?$AAe?$AA?$AA@ 00115a48     CEHWIntf.obj
 0002:0000335c       ??_7CHWIntf@@6B@           0011735c     HWIntf.obj
 0002:00003380       ??_7CriticalSection@@6B@   00117380     HWIntf.obj
 0002:0000464c       _GUID_b196b284_bab4_101a_b69c_00aa00341d07 0011864c     atlsd:atlfuncs.obj
 0002:0000465c       _GUID_00000000_0000_0000_c000_000000000046 0011865c     atlsd:atlfuncs.obj
 0002:00004670       ??_C@_1HA@FENMNPLO@?$AAf?$AA?3?$AA?2?$AAd?$AAd?$AA?2?$AAv?$AAc?$AAt?$AAo?$AAo?$AAl?$AAs?$AA?2?$AAv?$AAc?$AA7?$AAl?$AAi?$AAb?$AAs?$AAc?$AAe?$AA?2?$AAs?$AAh?$AAi?$AAp?$AA?2?$AAa?$AAt?$AAl@ 00118670     atlsd:atlfuncs.obj
 0002:000046e0       ??_C@_19LMDLLIGP@?$AAp?$AA?$DN?$AA?$DN?$AA0?$AA?$AA@ 001186e0     atlsd:atlfuncs.obj
 0002:000046ec       ??_C@_19JHCPJMAL@?$AAp?$AA?$CB?$AA?$DN?$AA0?$AA?$AA@ 001186ec     atlsd:atlfuncs.obj
 0002:000046f8       ??_C@_1HA@LPPEBACM@?$AAf?$AA?3?$AA?2?$AAd?$AAd?$AA?2?$AAv?$AAc?$AAt?$AAo?$AAo?$AAl?$AAs?$AA?2?$AAv?$AAc?$AA7?$AAl?$AAi?$AAb?$AAs?$AAc?$AAe?$AA?2?$AAs?$AAh?$AAi?$AAp?$AA?2?$AAa?$AAt?$AAl@ 001186f8     atlsd:atlfuncs.obj
 0002:00004768       ??_C@_1M@HLGKFCJM@?$AAf?$AAa?$AAl?$AAs?$AAe?$AA?$AA@ 00118768     atlsd:atlfuncs.obj
 0002:00004774       ??_C@_1CK@DFMKPFAK@?$AAA?$AAt?$AAl?$AAT?$AAh?$AAr?$AAo?$AAw?$AA?3?$AA?5?$AAh?$AAr?$AA?5?$AA?$DN?$AA?5?$AA0?$AAx?$AA?$CF?$AAx?$AA?6?$AA?$AA@ 00118774     atlsd:atlfuncs.obj
 0002:000047a0       ??_C@_0DI@MHBOGIL@f?3?2dd?2vctools?2vc7libsce?2ship?2atl@ 001187a0     atlsd:atlfuncs.obj
 0002:000047d8       ??_C@_1GM@IDLEHDFG@?$AAf?$AA?3?$AA?2?$AAd?$AAd?$AA?2?$AAv?$AAc?$AAt?$AAo?$AAo?$AAl?$AAs?$AA?2?$AAv?$AAc?$AA7?$AAl?$AAi?$AAb?$AAs?$AAc?$AAe?$AA?2?$AAs?$AAh?$AAi?$AAp?$AA?2?$AAa?$AAt?$AAl@ 001187d8     atlsd:atlfuncs.obj
 0002:00004844       ??_C@_1BE@NPGJNKLA@?$AAm?$AA_?$AAb?$AAL?$AAo?$AAc?$AAk?$AAe?$AAd?$AA?$AA@ 00118844     atlsd:atlfuncs.obj
 0002:00004858       ??_C@_1BG@OHCCAGNO@?$AA?$CB?$AAm?$AA_?$AAb?$AAL?$AAo?$AAc?$AAk?$AAe?$AAd?$AA?$AA@ 00118858     atlsd:atlfuncs.obj
 0002:00004870       ??_C@_1HE@LMFAHKHJ@?$AAf?$AA?3?$AA?2?$AAd?$AAd?$AA?2?$AAv?$AAc?$AAt?$AAo?$AAo?$AAl?$AAs?$AA?2?$AAv?$AAc?$AA7?$AAl?$AAi?$AAb?$AAs?$AAc?$AAe?$AA?2?$AAs?$AAh?$AAi?$AAp?$AA?2?$AAa?$AAt?$AAl@ 00118870     atlsd:atlfuncs.obj
 0002:00004a58       GUID_ATLVer30              00118a58     atlsd:atlbase.obj
 0002:00004a68       GUID_ATLVer70              00118a68     atlsd:atlbase.obj
 0002:00007d18       ??_C@_1JC@IHNNLNKC@?$AAf?$AA?3?$AA?2?$AAd?$AAd?$AA?2?$AAv?$AAc?$AAt?$AAo?$AAo?$AAl?$AAs?$AA?2?$AAv?$AAc?$AA7?$AAl?$AAi?$AAb?$AAs?$AAc?$AAe?$AA?2?$AAs?$AAh?$AAi?$AAp?$AA?2?$AAa?$AAt?$AAl@ 0011bd18     atlsd:Allocate.obj
 0002:00007dac       ??_C@_1BK@GFEAMNLJ@?$AAn?$AAC?$AAo?$AAo?$AAk?$AAi?$AAe?$AA?5?$AA?$CB?$AA?$DN?$AA?5?$AA0?$AA?$AA@ 0011bdac     atlsd:Allocate.obj
 0002:000081ac       ??_C@_17LGKOMLJ@?$AA?4?$AA?4?$AA?4?$AA?$AA@ 0011c1ac     LIBCMTD:dbgrpt.obj
 0002:000081b4       ??_C@_1CC@CGHMNGDG@?$AAA?$AAs?$AAs?$AAe?$AAr?$AAt?$AAi?$AAo?$AAn?$AA?5?$AAF?$AAa?$AAi?$AAl?$AAe?$AAd?$AA?$AA@ 0011c1b4     LIBCMTD:dbgrpt.obj
 0002:000081d8       ??_C@_1M@ILHOPKA@?$AAE?$AAr?$AAr?$AAo?$AAr?$AA?$AA@ 0011c1d8     LIBCMTD:dbgrpt.obj
 0002:000081e4       ??_C@_1BA@GLMCNLEM@?$AAW?$AAa?$AAr?$AAn?$AAi?$AAn?$AAg?$AA?$AA@ 0011c1e4     LIBCMTD:dbgrpt.obj
 0002:000081f8       ??_C@_1FC@DDJKODKC@?$AAf?$AA?3?$AA?2?$AAs?$AAp?$AA?2?$AAv?$AAc?$AAt?$AAo?$AAo?$AAl?$AAs?$AA?2?$AAc?$AAr?$AAt?$AAc?$AAe?$AA?2?$AAc?$AAr?$AAt?$AAw?$AA3?$AA2?$AA?2?$AAm?$AAi?$AAs?$AAc?$AA?2@ 0011c1f8     LIBCMTD:dbgrpt.obj
 0002:00008250       ??_C@_1EG@PEOEAKBB@?$AAM?$AAi?$AAc?$AAr?$AAo?$AAs?$AAo?$AAf?$AAt?$AA?5?$AAV?$AAi?$AAs?$AAu?$AAa?$AAl?$AA?5?$AAC?$AA?$CL?$AA?$CL?$AA?5?$AAD?$AAe?$AAb?$AAu?$AAg?$AA?5?$AAL?$AAi?$AAb?$AAr?$AAa@ 0011c250     LIBCMTD:dbgrpt.obj
 0002:00008298       ??_C@_1JI@EACPGHID@?$AAw?$AAc?$AAs?$AAc?$AAp?$AAy?$AA_?$AAs?$AA?$CI?$AAs?$AAz?$AAO?$AAu?$AAt?$AAM?$AAe?$AAs?$AAs?$AAa?$AAg?$AAe?$AA?0?$AA?5?$AA4?$AA0?$AA9?$AA6?$AA?0?$AA?5?$AAL?$AA?$CC?$AA_@ 0011c298     LIBCMTD:dbgrpt.obj
 0002:00008330       ??_C@_1FG@BBOLDHGF@?$AA_?$AAC?$AAr?$AAt?$AAD?$AAb?$AAg?$AAR?$AAe?$AAp?$AAo?$AAr?$AAt?$AA?3?$AA?5?$AAS?$AAt?$AAr?$AAi?$AAn?$AAg?$AA?5?$AAt?$AAo?$AAo?$AA?5?$AAl?$AAo?$AAn?$AAg?$AA?5?$AAo@ 0011c330     LIBCMTD:dbgrpt.obj
 0002:00008388       ??_C@_1KG@MFHGLLO@?$AAD?$AAe?$AAb?$AAu?$AAg?$AA?5?$AA?$CF?$AAs?$AA?$CB?$AA?6?$AA?6?$AAP?$AAr?$AAo?$AAg?$AAr?$AAa?$AAm?$AA?3?$AA?5?$AA?$CF?$AAs?$AA?$CF?$AAs?$AA?$CF?$AAs?$AA?$CF?$AAs?$AA?$CF?$AAs?$AA?$CF?$AAs@ 0011c388     LIBCMTD:dbgrpt.obj
 0002:00008430       ??_C@_1BE@CGCJKGHI@?$AA?6?$AAM?$AAo?$AAd?$AAu?$AAl?$AAe?$AA?3?$AA?5?$AA?$AA@ 0011c430     LIBCMTD:dbgrpt.obj
 0002:00008444       ??_C@_1BA@LNHECFIM@?$AA?6?$AAF?$AAi?$AAl?$AAe?$AA?3?$AA?5?$AA?$AA@ 0011c444     LIBCMTD:dbgrpt.obj
 0002:00008454       ??_C@_1BA@GLLGCPCK@?$AA?6?$AAL?$AAi?$AAn?$AAe?$AA?3?$AA?5?$AA?$AA@ 0011c454     LIBCMTD:dbgrpt.obj
 0002:00008464       ??_C@_13LBAGMAIH@?$AA?6?$AA?$AA@ 0011c464     LIBCMTD:dbgrpt.obj
 0002:00008468       ??_C@_1BK@PEDCIPMA@?$AAE?$AAx?$AAp?$AAr?$AAe?$AAs?$AAs?$AAi?$AAo?$AAn?$AA?3?$AA?5?$AA?$AA@ 0011c468     LIBCMTD:dbgrpt.obj
 0002:00008484       ??_C@_11LOCGONAA@?$AA?$AA@ 0011c484     LIBCMTD:dbgrpt.obj
 0002:00008488       ??_C@_1JM@GKDPCMEA@?$AAw?$AAc?$AAs?$AAn?$AAc?$AAp?$AAy?$AA_?$AAs?$AA?$CI?$AAs?$AAz?$AAS?$AAh?$AAo?$AAr?$AAt?$AAP?$AAr?$AAo?$AAg?$AAN?$AAa?$AAm?$AAe?$AA?0?$AA?5?$AA2?$AA6?$AA0?$AA?5?$AA?9@ 0011c488     LIBCMTD:dbgrpt.obj
 0002:00008528       ??_C@_1GI@DEDNNLCI@?$AAw?$AAc?$AAs?$AAc?$AAp?$AAy?$AA_?$AAs?$AA?$CI?$AAs?$AAz?$AAE?$AAx?$AAe?$AAN?$AAa?$AAm?$AAe?$AA?0?$AA?5?$AA2?$AA6?$AA0?$AA?0?$AA?5?$AAL?$AA?$CC?$AA?$DM?$AAp?$AAr?$AAo?$AAg@ 0011c528     LIBCMTD:dbgrpt.obj
 0002:00008590       ??_C@_1CI@PGJIFDEK@?$AA_?$AA_?$AAc?$AAr?$AAt?$AAM?$AAe?$AAs?$AAs?$AAa?$AAg?$AAe?$AAW?$AAi?$AAn?$AAd?$AAo?$AAw?$AAW?$AA?$AA@ 0011c590     LIBCMTD:dbgrpt.obj
 0002:000085b8       ??_C@_1CO@EAEJAADC@?$AA?$DM?$AAp?$AAr?$AAo?$AAg?$AAr?$AAa?$AAm?$AA?5?$AAn?$AAa?$AAm?$AAe?$AA?5?$AAu?$AAn?$AAk?$AAn?$AAo?$AAw?$AAn?$AA?$DO?$AA?$AA@ 0011c5b8     LIBCMTD:dbgrpt.obj
 0002:000085e8       ??_C@_1CK@DDKKOLAN@?$AAs?$AAi?$AAz?$AAe?$AAI?$AAn?$AAB?$AAy?$AAt?$AAe?$AAs?$AA?5?$AA?$DO?$AA?$DN?$AA?5?$AAc?$AAo?$AAu?$AAn?$AAt?$AA?$AA@ 0011c5e8     LIBCMTD:memmove_s.obj
 0002:00008614       ??_C@_1BI@DCHLDCPP@?$AAs?$AAr?$AAc?$AA?5?$AA?$CB?$AA?$DN?$AA?5?$AAN?$AAU?$AAL?$AAL?$AA?$AA@ 0011c614     LIBCMTD:memmove_s.obj
 0002:0000862c       ??_C@_1BE@NMKKBGPA@?$AAm?$AAe?$AAm?$AAm?$AAo?$AAv?$AAe?$AA_?$AAs?$AA?$AA@ 0011c62c     LIBCMTD:memmove_s.obj
 0002:00008640       ??_C@_1FM@JMDLOEFB@?$AAf?$AA?3?$AA?2?$AAs?$AAp?$AA?2?$AAv?$AAc?$AAt?$AAo?$AAo?$AAl?$AAs?$AA?2?$AAc?$AAr?$AAt?$AAc?$AAe?$AA?2?$AAc?$AAr?$AAt?$AAw?$AA3?$AA2?$AA?2?$AAs?$AAt?$AAr?$AAi?$AAn@ 0011c640     LIBCMTD:memmove_s.obj
 0002:0000869c       ??_C@_1BI@GKKCBDMD@?$AAd?$AAs?$AAt?$AA?5?$AA?$CB?$AA?$DN?$AA?5?$AAN?$AAU?$AAL?$AAL?$AA?$AA@ 0011c69c     LIBCMTD:memmove_s.obj
 0002:000086b4       ??_C@_1DM@MADKGDLO@?$AA?$CI?$AAL?$AA?$CC?$AAB?$AAu?$AAf?$AAf?$AAe?$AAr?$AA?5?$AAi?$AAs?$AA?5?$AAt?$AAo?$AAo?$AA?5?$AAs?$AAm?$AAa?$AAl?$AAl?$AA?$CC?$AA?5?$AA?$CG?$AA?$CG?$AA?5?$AA0?$AA?$CJ?$AA?$AA@ 0011c6b4     LIBCMTD:wcscpy_s.obj
 0002:000086f0       ??_C@_1CI@HCPHDDLE@?$AAB?$AAu?$AAf?$AAf?$AAe?$AAr?$AA?5?$AAi?$AAs?$AA?5?$AAt?$AAo?$AAo?$AA?5?$AAs?$AAm?$AAa?$AAl?$AAl?$AA?$AA@ 0011c6f0     LIBCMTD:wcscpy_s.obj
 0002:00008718       ??_C@_1CG@OFBJMIGJ@?$AA?$CI?$AA?$CI?$AA?$CI?$AA_?$AAS?$AAr?$AAc?$AA?$CJ?$AA?$CJ?$AA?$CJ?$AA?5?$AA?$CB?$AA?$DN?$AA?5?$AAN?$AAU?$AAL?$AAL?$AA?$AA@ 0011c718     LIBCMTD:wcscpy_s.obj
 0002:00008740       ??_C@_1BC@KIONAFPO@?$AAw?$AAc?$AAs?$AAc?$AAp?$AAy?$AA_?$AAs?$AA?$AA@ 0011c740     LIBCMTD:wcscpy_s.obj
 0002:00008758       ??_C@_1FE@IPADLOPJ@?$AAf?$AA?3?$AA?2?$AAs?$AAp?$AA?2?$AAv?$AAc?$AAt?$AAo?$AAo?$AAl?$AAs?$AA?2?$AAc?$AAr?$AAt?$AAc?$AAe?$AA?2?$AAc?$AAr?$AAt?$AAw?$AA3?$AA2?$AA?2?$AAh?$AA?2?$AAt?$AAc?$AAs@ 0011c758     LIBCMTD:wcscpy_s.obj
 0002:000087b0       ??_C@_1FC@PFMLEHKI@?$AA?$CI?$AA?$CI?$AA_?$AAD?$AAs?$AAt?$AA?$CJ?$AA?$CJ?$AA?5?$AA?$CB?$AA?$DN?$AA?5?$AAN?$AAU?$AAL?$AAL?$AA?5?$AA?$CG?$AA?$CG?$AA?5?$AA?$CI?$AA?$CI?$AA_?$AAS?$AAi?$AAz?$AAe?$AAI?$AAn?$AAW?$AAo?$AAr@ 0011c7b0     LIBCMTD:wcscpy_s.obj
 0002:00008804       ??_C@_1BE@PMMBFFCC@?$AAw?$AAc?$AAs?$AAn?$AAc?$AAp?$AAy?$AA_?$AAs?$AA?$AA@ 0011c804     LIBCMTD:wcsncpy_s.obj
 0002:00008818       ??_C@_1FG@OHHBDIEA@?$AAf?$AA?3?$AA?2?$AAs?$AAp?$AA?2?$AAv?$AAc?$AAt?$AAo?$AAo?$AAl?$AAs?$AA?2?$AAc?$AAr?$AAt?$AAc?$AAe?$AA?2?$AAc?$AAr?$AAt?$AAw?$AA3?$AA2?$AA?2?$AAh?$AA?2?$AAt?$AAc?$AAs@ 0011c818     LIBCMTD:wcsncpy_s.obj
 0002:00008870       ??_C@_0BJ@IPHDMCNM@fatal?5error?5in?5_lock?5?$CD0?6?$AA@ 0011c870     LIBCMTD:mlock.obj
 0002:00008890       ??_C@_1FE@PLIBPAGC@?$AAf?$AA?3?$AA?2?$AAs?$AAp?$AA?2?$AAv?$AAc?$AAt?$AAo?$AAo?$AAl?$AAs?$AA?2?$AAc?$AAr?$AAt?$AAc?$AAe?$AA?2?$AAc?$AAr?$AAt?$AAw?$AA3?$AA2?$AA?2?$AAm?$AAi?$AAs?$AAc?$AA?2@ 0011c890     LIBCMTD:dbgrptt.obj
 0002:000088e8       ??_C@_1MA@LBAMNNOB@?$AAs?$AAt?$AAr?$AAc?$AAp?$AAy?$AA_?$AAs?$AA?$CI?$AAs?$AAz?$AAO?$AAu?$AAt?$AAM?$AAe?$AAs?$AAs?$AAa?$AAg?$AAe?$AA2?$AA?0?$AA?5?$AA4?$AA0?$AA9?$AA6?$AA?0?$AA?5?$AA?$CC?$AA_@ 0011c8e8     LIBCMTD:dbgrptt.obj
 0002:000089a8       ??_C@_0DP@GNPEPHJD@_CrtDbgReport?3?5String?5too?5long?5o@ 0011c9a8     LIBCMTD:dbgrptt.obj
 0002:000089e8       ??_C@_1FI@DBAIJPJE@?$AAw?$AAc?$AAs?$AAc?$AAp?$AAy?$AA_?$AAs?$AA?$CI?$AAs?$AAz?$AAO?$AAu?$AAt?$AAM?$AAe?$AAs?$AAs?$AAa?$AAg?$AAe?$AA?0?$AA?5?$AA4?$AA0?$AA9?$AA6?$AA?0?$AA?5?$AAs?$AAz?$AAL@ 0011c9e8     LIBCMTD:dbgrptt.obj
 0002:00008a40       ??_C@_1BI@JIDBEPIG@?$AA?$CF?$AAs?$AA?$CI?$AA?$CF?$AAd?$AA?$CJ?$AA?5?$AA?3?$AA?5?$AA?$CF?$AAs?$AA?$AA@ 0011ca40     LIBCMTD:dbgrptt.obj
 0002:00008a58       ??_C@_1EK@PHCBEDKB@?$AAw?$AAc?$AAs?$AAc?$AAa?$AAt?$AA_?$AAs?$AA?$CI?$AAs?$AAz?$AAL?$AAi?$AAn?$AAe?$AAM?$AAe?$AAs?$AAs?$AAa?$AAg?$AAe?$AA?0?$AA?5?$AA4?$AA0?$AA9?$AA6?$AA?0?$AA?5?$AAL?$AA?$CC@ 0011ca58     LIBCMTD:dbgrptt.obj
 0002:00008aa8       ??_C@_1EK@NMDFGHMF@?$AAw?$AAc?$AAs?$AAc?$AAa?$AAt?$AA_?$AAs?$AA?$CI?$AAs?$AAz?$AAL?$AAi?$AAn?$AAe?$AAM?$AAe?$AAs?$AAs?$AAa?$AAg?$AAe?$AA?0?$AA?5?$AA4?$AA0?$AA9?$AA6?$AA?0?$AA?5?$AAL?$AA?$CC@ 0011caa8     LIBCMTD:dbgrptt.obj
 0002:00008af4       ??_C@_13CMNBPIDO@?$AA?$AN?$AA?$AA@ 0011caf4     LIBCMTD:dbgrptt.obj
 0002:00008af8       ??_C@_1FK@HPADHBBD@?$AAw?$AAc?$AAs?$AAc?$AAa?$AAt?$AA_?$AAs?$AA?$CI?$AAs?$AAz?$AAL?$AAi?$AAn?$AAe?$AAM?$AAe?$AAs?$AAs?$AAa?$AAg?$AAe?$AA?0?$AA?5?$AA4?$AA0?$AA9?$AA6?$AA?0?$AA?5?$AAs?$AAz@ 0011caf8     LIBCMTD:dbgrptt.obj
 0002:00008b58       ??_C@_1KO@DGAHENCH@?$AAw?$AAc?$AAs?$AAc?$AAp?$AAy?$AA_?$AAs?$AA?$CI?$AAs?$AAz?$AAL?$AAi?$AAn?$AAe?$AAM?$AAe?$AAs?$AAs?$AAa?$AAg?$AAe?$AA?0?$AA?5?$AA4?$AA0?$AA9?$AA6?$AA?0?$AA?5?$AAs?$AAz@ 0011cb58     LIBCMTD:dbgrptt.obj
 0002:00008c08       ??_C@_1CE@OJBNHDMO@?$AAA?$AAs?$AAs?$AAe?$AAr?$AAt?$AAi?$AAo?$AAn?$AA?5?$AAf?$AAa?$AAi?$AAl?$AAe?$AAd?$AA?$CB?$AA?$AA@ 0011cc08     LIBCMTD:dbgrptt.obj
 0002:00008c2c       ??_C@_1CG@FFFGGODN@?$AAA?$AAs?$AAs?$AAe?$AAr?$AAt?$AAi?$AAo?$AAn?$AA?5?$AAf?$AAa?$AAi?$AAl?$AAe?$AAd?$AA?3?$AA?5?$AA?$AA@ 0011cc2c     LIBCMTD:dbgrptt.obj
 0002:00008c58       ??_C@_1JK@KHFABAEO@?$AAw?$AAc?$AAs?$AAc?$AAp?$AAy?$AA_?$AAs?$AA?$CI?$AAs?$AAz?$AAU?$AAs?$AAe?$AAr?$AAM?$AAe?$AAs?$AAs?$AAa?$AAg?$AAe?$AA?0?$AA?5?$AA4?$AA0?$AA9?$AA6?$AA?0?$AA?5?$AAL?$AA?$CC@ 0011cc58     LIBCMTD:dbgrptt.obj
 0002:00008cf4       ??_C@_1BA@ELMMDCFC@?$AA?0?$AA?5?$AAL?$AAi?$AAn?$AAe?$AA?5?$AA?$AA@ 0011ccf4     LIBCMTD:dbgrptt.obj
 0002:00008d04       ??_C@_1BO@OCHMLCAG@?$AA?$DM?$AAf?$AAi?$AAl?$AAe?$AA?5?$AAu?$AAn?$AAk?$AAn?$AAo?$AAw?$AAn?$AA?$DO?$AA?$AA@ 0011cd04     LIBCMTD:dbgrptt.obj
 0002:00008d28       ??_C@_1EM@MJFLEDMB@?$AAS?$AAe?$AAc?$AAo?$AAn?$AAd?$AA?5?$AAC?$AAh?$AAa?$AAn?$AAc?$AAe?$AA?5?$AAA?$AAs?$AAs?$AAe?$AAr?$AAt?$AAi?$AAo?$AAn?$AA?5?$AAF?$AAa?$AAi?$AAl?$AAe?$AAd?$AA?3?$AA?5@ 0011cd28     LIBCMTD:dbgrptt.obj
 0002:00008d78       ??_C@_1FA@CNLLOMHI@?$AA_?$AAi?$AAt?$AAo?$AAw?$AA_?$AAs?$AA?$CI?$AAn?$AAL?$AAi?$AAn?$AAe?$AA?0?$AA?5?$AAs?$AAz?$AAL?$AAi?$AAn?$AAe?$AAM?$AAe?$AAs?$AAs?$AAa?$AAg?$AAe?$AA?0?$AA?5?$AA4?$AA0@ 0011cd78     LIBCMTD:dbgrptt.obj
 0002:00008dc8       ??_C@_1CA@HPALHDOD@?$AA_?$AAV?$AAC?$AAr?$AAt?$AAD?$AAb?$AAg?$AAR?$AAe?$AAp?$AAo?$AAr?$AAt?$AAW?$AA?$AA@ 0011cdc8     LIBCMTD:dbgrptt.obj
 0002:00008de8       ??_C@_1CG@MKBKDNCP@?$AAG?$AAe?$AAt?$AAL?$AAa?$AAs?$AAt?$AAA?$AAc?$AAt?$AAi?$AAv?$AAe?$AAP?$AAo?$AAp?$AAu?$AAp?$AA?$AA@ 0011cde8     LIBCMTD:crtmbox.obj
 0002:00008e10       ??_C@_1CA@HNKPMKAN@?$AAG?$AAe?$AAt?$AAA?$AAc?$AAt?$AAi?$AAv?$AAe?$AAW?$AAi?$AAn?$AAd?$AAo?$AAw?$AA?$AA@ 0011ce10     LIBCMTD:crtmbox.obj
 0002:00008e30       ??_C@_1BI@OGPGOOGK@?$AAM?$AAe?$AAs?$AAs?$AAa?$AAg?$AAe?$AAB?$AAo?$AAx?$AAW?$AA?$AA@ 0011ce30     LIBCMTD:crtmbox.obj
 0002:00008e48       ??_C@_1BI@IENOMFML@?$AAC?$AAO?$AAR?$AAE?$AAD?$AAL?$AAL?$AA?4?$AAD?$AAL?$AAL?$AA?$AA@ 0011ce48     LIBCMTD:crtmbox.obj
 0002:00008e60       ??_C@_1BC@CFJEPFGF@?$AAs?$AAt?$AAr?$AAc?$AAp?$AAy?$AA_?$AAs?$AA?$AA@ 0011ce60     LIBCMTD:strcpy_s.obj
 0002:00008e78       ??_C@_1FC@NCPEPIBI@?$AA?$CI?$AA?$CI?$AA_?$AAD?$AAs?$AAt?$AA?$CJ?$AA?$CJ?$AA?5?$AA?$CB?$AA?$DN?$AA?5?$AAN?$AAU?$AAL?$AAL?$AA?5?$AA?$CG?$AA?$CG?$AA?5?$AA?$CI?$AA?$CI?$AA_?$AAS?$AAi?$AAz?$AAe?$AAI?$AAn?$AAB?$AAy?$AAt@ 0011ce78     LIBCMTD:strcpy_s.obj
 0002:00008ed0       ??_C@_1FA@MJKDNFFB@?$AA?$CI?$AAL?$AA?$CC?$AAS?$AAt?$AAr?$AAi?$AAn?$AAg?$AA?5?$AAi?$AAs?$AA?5?$AAn?$AAo?$AAt?$AA?5?$AAn?$AAu?$AAl?$AAl?$AA?5?$AAt?$AAe?$AAr?$AAm?$AAi?$AAn?$AAa?$AAt?$AAe?$AAd@ 0011ced0     LIBCMTD:wcscat_s.obj
 0002:00008f20       ??_C@_1DM@FHLMIEG@?$AAS?$AAt?$AAr?$AAi?$AAn?$AAg?$AA?5?$AAi?$AAs?$AA?5?$AAn?$AAo?$AAt?$AA?5?$AAn?$AAu?$AAl?$AAl?$AA?5?$AAt?$AAe?$AAr?$AAm?$AAi?$AAn?$AAa?$AAt?$AAe?$AAd?$AA?$AA@ 0011cf20     LIBCMTD:wcscat_s.obj
 0002:00008f5c       ??_C@_1BC@PLIEPKPJ@?$AAw?$AAc?$AAs?$AAc?$AAa?$AAt?$AA_?$AAs?$AA?$AA@ 0011cf5c     LIBCMTD:wcscat_s.obj
 0002:00008f70       ??_C@_1FE@EHLIBGFJ@?$AAf?$AA?3?$AA?2?$AAs?$AAp?$AA?2?$AAv?$AAc?$AAt?$AAo?$AAo?$AAl?$AAs?$AA?2?$AAc?$AAr?$AAt?$AAc?$AAe?$AA?2?$AAc?$AAr?$AAt?$AAw?$AA3?$AA2?$AA?2?$AAh?$AA?2?$AAt?$AAc?$AAs@ 0011cf70     LIBCMTD:wcscat_s.obj
 0002:00008fc4       ??_C@_1CM@HABGDNLJ@?$AAl?$AAe?$AAn?$AAg?$AAt?$AAh?$AA?5?$AA?$DM?$AA?5?$AAs?$AAi?$AAz?$AAe?$AAI?$AAn?$AAT?$AAC?$AAh?$AAa?$AAr?$AAs?$AA?$AA@ 0011cfc4     LIBCMTD:xtows.obj
 0002:00008ff0       ??_C@_1DE@PCJGDBBD@?$AA2?$AA?5?$AA?$DM?$AA?$DN?$AA?5?$AAr?$AAa?$AAd?$AAi?$AAx?$AA?5?$AA?$CG?$AA?$CG?$AA?5?$AAr?$AAa?$AAd?$AAi?$AAx?$AA?5?$AA?$DM?$AA?$DN?$AA?5?$AA3?$AA6?$AA?$AA@ 0011cff0     LIBCMTD:xtows.obj
 0002:00009028       ??_C@_1FA@MKGGAGEI@?$AAs?$AAi?$AAz?$AAe?$AAI?$AAn?$AAT?$AAC?$AAh?$AAa?$AAr?$AAs?$AA?5?$AA?$DO?$AA?5?$AA?$CI?$AAs?$AAi?$AAz?$AAe?$AA_?$AAt?$AA?$CJ?$AA?$CI?$AAi?$AAs?$AA_?$AAn?$AAe?$AAg?$AA?5?$AA?$DP@ 0011d028     LIBCMTD:xtows.obj
 0002:00009078       ??_C@_1CC@JNJFIMGE@?$AAs?$AAi?$AAz?$AAe?$AAI?$AAn?$AAT?$AAC?$AAh?$AAa?$AAr?$AAs?$AA?5?$AA?$DO?$AA?5?$AA0?$AA?$AA@ 0011d078     LIBCMTD:xtows.obj
 0002:0000909c       ??_C@_1O@NCBFODOE@?$AAx?$AAt?$AAo?$AAw?$AA_?$AAs?$AA?$AA@ 0011d09c     LIBCMTD:xtows.obj
 0002:000090b0       ??_C@_1FE@LAGNOOBA@?$AAf?$AA?3?$AA?2?$AAs?$AAp?$AA?2?$AAv?$AAc?$AAt?$AAo?$AAo?$AAl?$AAs?$AA?2?$AAc?$AAr?$AAt?$AAc?$AAe?$AA?2?$AAc?$AAr?$AAt?$AAw?$AA3?$AA2?$AA?2?$AAc?$AAo?$AAn?$AAv?$AAe@ 0011d0b0     LIBCMTD:xtows.obj
 0002:00009104       ??_C@_1BI@ICGGMGLK@?$AAb?$AAu?$AAf?$AA?5?$AA?$CB?$AA?$DN?$AA?5?$AAN?$AAU?$AAL?$AAL?$AA?$AA@ 0011d104     LIBCMTD:xtows.obj
 0002:0000911c       IID_IPersistStream         0011d11c     uuid:objidl_i_guid12.obj
 0002:0000926c       _TI1?AVCAtlException@ATL@@ 0011d26c     atlsd:Externs.obj
 0002:0000927c       _CTA1?AVCAtlException@ATL@@ 0011d27c     atlsd:Externs.obj
 0002:00009284       _CT??_R0?AVCAtlException@ATL@@@84 0011d284     atlsd:Externs.obj
 0002:000092a0       __IMPORT_DESCRIPTOR_sw_utilityG 0011d2a0     sw_utilityG:sw_utilityG.dll
 0002:000092b4       __IMPORT_DESCRIPTOR_COREDLL 0011d2b4     coredll:COREDLL.dll
 0002:000092c8       __IMPORT_DESCRIPTOR_ole32  0011d2c8     ole32:ole32.dll
 0002:000092dc       __NULL_IMPORT_DESCRIPTOR   0011d2dc     sw_utilityG:sw_utilityG.dll
 0003:00000000       __imp___security_gen_cookie 0011e000     coredll:COREDLL.dll
 0003:00000004       __imp_InterlockedCompareExchange 0011e004     coredll:COREDLL.dll
 0003:00000008       __imp_TlsGetValue          0011e008     coredll:COREDLL.dll
 0003:0000000c       __imp_TlsSetValue          0011e00c     coredll:COREDLL.dll
 0003:00000010       __imp_malloc               0011e010     coredll:COREDLL.dll
 0003:00000014       __imp_TerminateProcess     0011e014     coredll:COREDLL.dll
 0003:00000018       __imp_SetLastError         0011e018     coredll:COREDLL.dll
 0003:0000001c       __imp_wcstombs             0011e01c     coredll:COREDLL.dll
 0003:00000020       __imp_WriteFile            0011e020     coredll:COREDLL.dll
 0003:00000024       __imp_??3@YAXPAX@Z         0011e024     coredll:COREDLL.dll
 0003:00000028       __imp_Sleep                0011e028     coredll:COREDLL.dll
 0003:0000002c       __imp_GetProcAddressW      0011e02c     coredll:COREDLL.dll
 0003:00000030       __imp_LoadLibraryW         0011e030     coredll:COREDLL.dll
 0003:00000034       __imp_wcscpy               0011e034     coredll:COREDLL.dll
 0003:00000038       __imp_memset               0011e038     coredll:COREDLL.dll
 0003:0000003c       __imp_FreeLibrary          0011e03c     coredll:COREDLL.dll
 0003:00000040       __imp__snprintf            0011e040     coredll:COREDLL.dll
 0003:00000044       __imp_NKDbgPrintfW         0011e044     coredll:COREDLL.dll
 0003:00000048       __imp_WaitForSingleObject  0011e048     coredll:COREDLL.dll
 0003:0000004c       __imp_DeleteCriticalSection 0011e04c     coredll:COREDLL.dll
 0003:00000050       __imp_free                 0011e050     coredll:COREDLL.dll
 0003:00000054       __imp_RaiseException       0011e054     coredll:COREDLL.dll
 0003:00000058       __imp_CreateEventW         0011e058     coredll:COREDLL.dll
 0003:0000005c       __imp__purecall            0011e05c     coredll:COREDLL.dll
 0003:00000060       __imp_InitializeCriticalSection 0011e060     coredll:COREDLL.dll
 0003:00000064       __imp_CloseHandle          0011e064     coredll:COREDLL.dll
 0003:00000068       __imp_EnterCriticalSection 0011e068     coredll:COREDLL.dll
 0003:0000006c       __imp_LeaveCriticalSection 0011e06c     coredll:COREDLL.dll
 0003:00000070       __imp___rt_udiv            0011e070     coredll:COREDLL.dll
 0003:00000074       __imp_WaitForMultipleObjects 0011e074     coredll:COREDLL.dll
 0003:00000078       __imp_GetTickCount         0011e078     coredll:COREDLL.dll
 0003:0000007c       __imp_EventModify          0011e07c     coredll:COREDLL.dll
 0003:00000080       __imp_DisableThreadLibraryCalls 0011e080     coredll:COREDLL.dll
 0003:00000084       __imp_GetModuleFileNameW   0011e084     coredll:COREDLL.dll
 0003:00000088       __imp_??2@YAPAXI@Z         0011e088     coredll:COREDLL.dll
 0003:0000008c       __imp_CreateThread         0011e08c     coredll:COREDLL.dll
 0003:00000090       __imp___report_gsfailure   0011e090     coredll:COREDLL.dll
 0003:00000094       __imp_LocalReAlloc         0011e094     coredll:COREDLL.dll
 0003:00000098       __imp_LocalAlloc           0011e098     coredll:COREDLL.dll
 0003:0000009c       __imp_LocalSize            0011e09c     coredll:COREDLL.dll
 0003:000000a0       __imp_LocalFree            0011e0a0     coredll:COREDLL.dll
 0003:000000a4       __imp_memmove              0011e0a4     coredll:COREDLL.dll
 0003:000000a8       __imp_DispatchMessageW     0011e0a8     coredll:COREDLL.dll
 0003:000000ac       __imp_TranslateMessage     0011e0ac     coredll:COREDLL.dll
 0003:000000b0       __imp_GetMessageW          0011e0b0     coredll:COREDLL.dll
 0003:000000b4       __imp_PeekMessageW         0011e0b4     coredll:COREDLL.dll
 0003:000000b8       __imp_MsgWaitForMultipleObjectsEx 0011e0b8     coredll:COREDLL.dll
 0003:000000bc       __imp___C_specific_handler 0011e0bc     coredll:COREDLL.dll
 0003:000000c0       __imp_GetModuleHandleW     0011e0c0     coredll:COREDLL.dll
 0003:000000c4       __imp_realloc              0011e0c4     coredll:COREDLL.dll
 0003:000000c8       __imp__snwprintf           0011e0c8     coredll:COREDLL.dll
 0003:000000cc       __imp_memcpy               0011e0cc     coredll:COREDLL.dll
 0003:000000d0       __imp___CxxThrowException  0011e0d0     coredll:COREDLL.dll
 0003:000000d4       __imp_??_7type_info@@6B@   0011e0d4     coredll:COREDLL.dll
 0003:000000d8       __imp_OpenEventW           0011e0d8     coredll:COREDLL.dll
 0003:000000dc       __imp_OutputDebugStringW   0011e0dc     coredll:COREDLL.dll
 0003:000000e0       __imp__vsnwprintf          0011e0e0     coredll:COREDLL.dll
 0003:000000e4       __imp_VirtualAlloc         0011e0e4     coredll:COREDLL.dll
 0003:000000e8       __imp_UnmapViewOfFile      0011e0e8     coredll:COREDLL.dll
 0003:000000ec       __imp_memcmp               0011e0ec     coredll:COREDLL.dll
 0003:000000f0       __imp_GetSystemInfo        0011e0f0     coredll:COREDLL.dll
 0003:000000f4       __imp_MapViewOfFile        0011e0f4     coredll:COREDLL.dll
 0003:000000f8       __imp_GetLastError         0011e0f8     coredll:COREDLL.dll
 0003:000000fc       __imp_CreateFileMappingW   0011e0fc     coredll:COREDLL.dll
 0003:00000100       __imp__wcsicmp             0011e100     coredll:COREDLL.dll
 0003:00000104       __imp_InterlockedIncrement 0011e104     coredll:COREDLL.dll
 0003:00000108       __imp_InterlockedDecrement 0011e108     coredll:COREDLL.dll
 0003:0000010c       __imp_wcslen               0011e10c     coredll:COREDLL.dll
 0003:00000110       __imp_strcmp               0011e110     coredll:COREDLL.dll
 0003:00000114       __imp_?terminate@std@@YAXXZ 0011e114     coredll:COREDLL.dll
 0003:00000118       __imp_TlsCall              0011e118     coredll:COREDLL.dll
 0003:0000011c       \177COREDLL_NULL_THUNK_DATA 0011e11c     coredll:COREDLL.dll
 0003:00000120       __imp_WriteClassStm        0011e120     ole32:ole32.dll
 0003:00000124       __imp_CoCreateInstance     0011e124     ole32:ole32.dll
 0003:00000128       __imp_ReadClassStm         0011e128     ole32:ole32.dll
 0003:0000012c       __imp_CreateStreamOnHGlobal 0011e12c     ole32:ole32.dll
 0003:00000130       \177ole32_NULL_THUNK_DATA  0011e130     ole32:ole32.dll
 0003:00000134       __imp_?GetRegValue@@YAJPAUHKEY__@@PBG1AAK@Z 0011e134     sw_utilityG:sw_utilityG.dll
 0003:00000138       __imp_?SetRegValue@@YAJPAUHKEY__@@PBG1K@Z 0011e138     sw_utilityG:sw_utilityG.dll
 0003:0000013c       __imp_?SWAI_GetRegValue@@YAJPAUHKEY__@@PBG1PAGPAK@Z 0011e13c     sw_utilityG:sw_utilityG.dll
 0003:00000140       __imp_?LogC@@YAXPBGZZ      0011e140     sw_utilityG:sw_utilityG.dll
 0003:00000144       __imp_?SWAI_GetRegValue@@YAJPAUHKEY__@@PBG1AAK@Z 0011e144     sw_utilityG:sw_utilityG.dll
 0003:00000148       __imp_?LogStoreFileLine@@YAXPAGH@Z 0011e148     sw_utilityG:sw_utilityG.dll
 0003:0000014c       __imp_?LogW@@YAXPBGZZ      0011e14c     sw_utilityG:sw_utilityG.dll
 0003:00000150       __imp_?WriteLog@@YAXKPBGZZ 0011e150     sw_utilityG:sw_utilityG.dll
 0003:00000154       \177sw_utilityG_NULL_THUNK_DATA 0011e154     sw_utilityG:sw_utilityG.dll
 0003:00000158       __xc_a                     0011e158     corelibc:crt0init.obj
 0003:000001cc       __xc_z                     0011e1cc     corelibc:crt0init.obj
 0003:000001d0       __xi_a                     0011e1d0     corelibc:crt0init.obj
 0003:000001d4       __xi_z                     0011e1d4     corelibc:crt0init.obj
 0003:000001d8       __xp_a                     0011e1d8     corelibc:crt0init.obj
 0003:000001dc       __xp_z                     0011e1dc     corelibc:crt0init.obj
 0003:000001e0       __xt_a                     0011e1e0     corelibc:crt0init.obj
 0003:000001e4       __xt_z                     0011e1e4     corelibc:crt0init.obj
 0003:000001e8       ?HW2SWNotificationPowerMode@@3PAHA 0011e1e8     HWIntf.obj
 0003:000001fc       __security_cookie_complement 0011e1fc     corelibc:seccook.obj
 0003:00000200       __security_cookie          0011e200     corelibc:seccook.obj
 0003:00000204       _pRawDllMain               0011e204     atlsd:atlbase.obj
 0003:00000208       ?g_pszUpdateEventName@@3PB_WB 0011e208     atlsd:Externs.obj
 0003:0000020c       ?g_pszAllocFileMapName@@3PB_WB 0011e20c     atlsd:Externs.obj
 0003:00000210       ?g_pszKernelObjFmt@@3PB_WB 0011e210     atlsd:Externs.obj
 0003:00000214       ??_R0?AVCAtlException@ATL@@@8 0011e214     atlsd:Externs.obj
 0003:00000368       _crtAssertBusy             0011e368     LIBCMTD:dbgrptt.obj
 0003:0000036c       _CrtDbgMode                0011e36c     LIBCMTD:dbgrptt.obj
 0003:00000378       _CrtDbgFile                0011e378     LIBCMTD:dbgrptt.obj
 0003:00000384       _aexit_rtn                 0011e384     LIBCMTD:crt0dat.obj
 0003:00000388       ?m_bInitFailed@CAtlBaseModule@ATL@@2_NA 0011e388     CEHWIntf.obj
 0003:0000038c       ?thePwrCtrlObj@@3PAVCCEHWIntf@@A 0011e38c     CEHWIntf.obj
 0003:00000390       ?g_ModuleName@@3PAGA       0011e390     SwiHWAux.obj
 0003:0000059c       ?theHWIntf@@3PAVCCEHWIntf@@A 0011e59c     SwiHWAux.obj
 0003:000005a0       ?g_hinstThisDll@@3PAXA     0011e5a0     SwiHWAux.obj
 0003:000005a4       ?g_IsCriticalPower@@3HA    0011e5a4     SwiHWAux.obj
 0003:000005a8       ?gCallBackP@@3P6AXPAUSwiNotifyVariant@@@ZA 0011e5a8     SwiHWAux.obj
 0003:000005ac       ?theSWIHWCR@@3VCriticalSection@@A 0011e5ac     SwiHWAux.obj
 0003:000005c4       ?_pAtlRawDllMain@@3P6AHPAXK0@ZA 0011e5c4     atlsd:atlbase.obj
 0003:000005c8       ?_AtlModuleInstance@ATL@@3PAUHINSTANCE__@@A 0011e5c8     atlsd:atlbase.obj
 0003:000005cc       ?_AtlBaseModule@ATL@@3VCAtlBaseModule@1@A 0011e5cc     atlsd:atlbase.obj
 0003:00000650       ?atlTraceGeneral@ATL@@3VCTraceCategory@1@A 0011e650     atlsd:atltrace.obj
 0003:00000654       ?atlTraceCOM@ATL@@3VCTraceCategory@1@A 0011e654     atlsd:atltrace.obj
 0003:00000658       ?atlTraceQI@ATL@@3VCTraceCategory@1@A 0011e658     atlsd:atltrace.obj
 0003:0000065c       ?atlTraceRegistrar@ATL@@3VCTraceCategory@1@A 0011e65c     atlsd:atltrace.obj
 0003:00000660       ?atlTraceRefcount@ATL@@3VCTraceCategory@1@A 0011e660     atlsd:atltrace.obj
 0003:00000664       ?atlTraceWindowing@ATL@@3VCTraceCategory@1@A 0011e664     atlsd:atltrace.obj
 0003:00000668       ?atlTraceControls@ATL@@3VCTraceCategory@1@A 0011e668     atlsd:atltrace.obj
 0003:0000066c       ?atlTraceHosting@ATL@@3VCTraceCategory@1@A 0011e66c     atlsd:atltrace.obj
 0003:00000670       ?atlTraceNotImpl@ATL@@3VCTraceCategory@1@A 0011e670     atlsd:atltrace.obj
 0003:00000674       ?atlTraceAllocation@ATL@@3VCTraceCategory@1@A 0011e674     atlsd:atltrace.obj
 0003:00000678       ?atlTraceException@ATL@@3VCTraceCategory@1@A 0011e678     atlsd:atltrace.obj
 0003:0000067c       ?atlTraceTime@ATL@@3VCTraceCategory@1@A 0011e67c     atlsd:atltrace.obj
 0003:00000680       ?atlTraceCache@ATL@@3VCTraceCategory@1@A 0011e680     atlsd:atltrace.obj
 0003:00000684       ?atlTraceStencil@ATL@@3VCTraceCategory@1@A 0011e684     atlsd:atltrace.obj
 0003:00000688       ?atlTraceString@ATL@@3VCTraceCategory@1@A 0011e688     atlsd:atltrace.obj
 0003:0000068c       ?atlTraceMap@ATL@@3VCTraceCategory@1@A 0011e68c     atlsd:atltrace.obj
 0003:00000690       ?atlTraceUtil@ATL@@3VCTraceCategory@1@A 0011e690     atlsd:atltrace.obj
 0003:00000694       ?atlTraceSync@ATL@@3VCTraceCategory@1@A 0011e694     atlsd:atltrace.obj
 0003:00000698       ?atlTraceUser@ATL@@3VCTraceCategory@1@A 0011e698     atlsd:atltrace.obj
 0003:0000069c       ?atlTraceUser2@ATL@@3VCTraceCategory@1@A 0011e69c     atlsd:atltrace.obj
 0003:000006a0       ?atlTraceUser3@ATL@@3VCTraceCategory@1@A 0011e6a0     atlsd:atltrace.obj
 0003:000006a4       ?atlTraceUser4@ATL@@3VCTraceCategory@1@A 0011e6a4     atlsd:atltrace.obj
 0003:000006a8       ?g_Allocator@@3VCAtlAllocator@@A 0011e6a8     atlsd:Externs.obj
 0003:000006dc       ?s_trace@CTrace@ATL@@2V12@A 0011e6dc     atlsd:Externs.obj
 0003:00000830       __onexitend                0011e830     <common>
 0003:00000834       __onexitbegin              0011e834     <common>
 0003:00000838       _exitflag                  0011e838     <common>
 0003:0000083c       _pfnReportHook             0011e83c     <common>
 0003:00000840       _pReportHookListW          0011e840     <common>
 0003:00000844       _pReportHookList           0011e844     <common>

 entry point at        0001:00003938

 Static symbols

 0001:00000274       __unwind$58910             00101274 f   CEHWIntf.obj
 0001:00000324       __unwind$58954             00101324 f   CEHWIntf.obj
 0001:0000185c       __unwind$40395             0010285c f   HWIntf.obj
 0001:00001bf8       __unwind$40473             00102bf8 f   HWIntf.obj
 0001:00002420       __unwind$40497             00103420 f   HWIntf.obj
 0001:00003b68       doexit                     00104b68 f   corelibc:crt0dat.obj
 0001:00006314       ?_ATLLoadOle32API@ATL@@YAP6AHXZPB_W@Z 00107314 f   atlsd:atlbase.obj
 0001:00007d7c       ?Init@@YA_NXZ              00108d7c f   atlsd:Externs.obj
 0001:00009cf8       ?ShouldTraceOutput@ATL@@YA_NKKIPAPBVCAtlTraceCategory@@PAP6AHHPB_WH11ZZ@Z 0010acf8 f   atlsd:AtlDebugAPI.obj
 0001:0000ca44       ?FindHandler@@YAEPAUEHExceptionRecord@@PAKPAU_CONTEXT@@PAU_DISPATCHER_CONTEXT@@PBU_s_FuncInfo@@H@Z 0010da44 f   LIBCMTD:frame_ce.obj
 0001:0000d038       ?TypeMatch@@YAHPBU_s_HandlerType@@PBU_s_CatchableType@@PBU_s_ThrowInfo@@@Z 0010e038 f   LIBCMTD:frame_ce.obj
 0001:0000d3fc       ?FrameUnwindFilter@@YAHPAU_EXCEPTION_POINTERS@@@Z 0010e3fc f   LIBCMTD:frame_ce.obj
 0001:0000d488       ?CallCatchBlock@@YAPAXPAUEHExceptionRecord@@PAKPAU_CONTEXT@@PBU_s_FuncInfo@@PAXHK@Z 0010e488 f   LIBCMTD:frame_ce.obj
 0001:0000da24       ?CanThisExceptionObjectBeDestructed@@YAEPAUEHExceptionRecord@@E@Z 0010ea24 f   LIBCMTD:frame_ce.obj
 0001:0000dcb0       ?BuildCatchObject@@YAXPAUEHExceptionRecord@@PAKPBU_s_HandlerType@@PBU_s_CatchableType@@@Z 0010ecb0 f   LIBCMTD:frame_ce.obj
 0001:0000e000       ?AdjustPointer@@YAPAXPAXABUPMD@@@Z 0010f000 f   LIBCMTD:frame_ce.obj
 0001:0001109c       __crtInitCritSecNoSpinCount 0011209c f   LIBCMTD:initcrit.obj
 0001:00011c34       xtow_s                     00112c34 f   LIBCMTD:xtows.obj
 0001:00012570       ??__EtheSWIHWCR@@YAXXZ     00113570 f   SwiHWAux.obj
 0001:00012590       ??__E_AtlBaseModule@ATL@@YAXXZ 00113590 f   atlsd:atlbase.obj
 0001:000125cc       ??__EatlTraceGeneral@ATL@@YAXXZ 001135cc f   atlsd:atltrace.obj
 0001:000125fc       ??__EatlTraceCOM@ATL@@YAXXZ 001135fc f   atlsd:atltrace.obj
 0001:0001262c       ??__EatlTraceQI@ATL@@YAXXZ 0011362c f   atlsd:atltrace.obj
 0001:0001265c       ??__EatlTraceRegistrar@ATL@@YAXXZ 0011365c f   atlsd:atltrace.obj
 0001:0001268c       ??__EatlTraceRefcount@ATL@@YAXXZ 0011368c f   atlsd:atltrace.obj
 0001:000126bc       ??__EatlTraceWindowing@ATL@@YAXXZ 001136bc f   atlsd:atltrace.obj
 0001:000126ec       ??__EatlTraceControls@ATL@@YAXXZ 001136ec f   atlsd:atltrace.obj
 0001:0001271c       ??__EatlTraceHosting@ATL@@YAXXZ 0011371c f   atlsd:atltrace.obj
 0001:0001274c       ??__EatlTraceNotImpl@ATL@@YAXXZ 0011374c f   atlsd:atltrace.obj
 0001:0001277c       ??__EatlTraceAllocation@ATL@@YAXXZ 0011377c f   atlsd:atltrace.obj
 0001:000127ac       ??__EatlTraceException@ATL@@YAXXZ 001137ac f   atlsd:atltrace.obj
 0001:000127dc       ??__EatlTraceTime@ATL@@YAXXZ 001137dc f   atlsd:atltrace.obj
 0001:0001280c       ??__EatlTraceCache@ATL@@YAXXZ 0011380c f   atlsd:atltrace.obj
 0001:0001283c       ??__EatlTraceStencil@ATL@@YAXXZ 0011383c f   atlsd:atltrace.obj
 0001:0001286c       ??__EatlTraceString@ATL@@YAXXZ 0011386c f   atlsd:atltrace.obj
 0001:0001289c       ??__EatlTraceMap@ATL@@YAXXZ 0011389c f   atlsd:atltrace.obj
 0001:000128cc       ??__EatlTraceUtil@ATL@@YAXXZ 001138cc f   atlsd:atltrace.obj
 0001:000128fc       ??__EatlTraceSync@ATL@@YAXXZ 001138fc f   atlsd:atltrace.obj
 0001:0001292c       ??__EatlTraceUser@ATL@@YAXXZ 0011392c f   atlsd:atltrace.obj
 0001:0001295c       ??__EatlTraceUser2@ATL@@YAXXZ 0011395c f   atlsd:atltrace.obj
 0001:0001298c       ??__EatlTraceUser3@ATL@@YAXXZ 0011398c f   atlsd:atltrace.obj
 0001:000129bc       ??__EatlTraceUser4@ATL@@YAXXZ 001139bc f   atlsd:atltrace.obj
 0001:000129ec       ??__Eg_Allocator@@YAXXZ    001139ec f   atlsd:Externs.obj
 0001:00012a28       ??__Eg_bInitialized@@YAXXZ 00113a28 f   atlsd:Externs.obj
 0001:00012a60       ??__E?s_trace@CTrace@ATL@@2V12@A@@YAXXZ 00113a60 f   atlsd:Externs.obj
 0001:00012aa4       ??__FtheSWIHWCR@@YAXXZ     00113aa4 f   SwiHWAux.obj
 0001:00012ab8       ??__F_AtlBaseModule@ATL@@YAXXZ 00113ab8 f   atlsd:atlbase.obj
 0001:00012adc       ??__Fg_Allocator@@YAXXZ    00113adc f   atlsd:Externs.obj
 0001:00012b00       ??__F?s_trace@CTrace@ATL@@2V12@A@@YAXXZ 00113b00 f   atlsd:Externs.obj
